:040000000C948513C4
:040028000C942C5AAE
:040040000C94F359D0
:040048000C940F7293
:040050000C94B472E6
:14008C00F1B4F1B4F1B4F1B4F1B4F1B4F1B4F1B4D5B4E0B41B
:1400A00005B5F1B4F1B4F1B437C0E4C0E4C0E4C0E4C0E4C078
:1400B400E4C0E4C037C037C0EEBF37C037C007C055C055C076
:1400C80055C055C055C055C055C055C055C055C055C055C052
:1400DC0055C059C159C159C159C159C159C159C159C159C111
:1400F00059C159C159C159C1E5C231C331C331C331C331C329
:1401040031C331C3E5C2E5C2D8C2E5C2E5C2E5C2FFC2FFC2A0
:14011800FFC2FFC2FFC2FFC2FFC2FFC2FFC2FFC2FFC2FFC249
:14012C00FFC2F5D48BD363D663D6D0DBF7DBD0DB30DC69DCEC
:14014000F7DBA0DC30DC1CE343EA4FE667E60A0D4C697374F0
:14015400206F6620617661696C61626C652073657269616C41
:1401680020636F6D6D616E64733A0D0A0D0A48656C702020E0
:14017C002020202020202020202D2054686973204D656E75B5
:140190000D0A73657473657269616C2020202020202D20412A
:1401A4006C6C6F777320796F7520746F20636F6E666967758B
:1401B8007265207468652073657269616C20706F72740D0A5F
:1401CC003F69702020202020202020202020202D205072690F
:1401E0006E7473207468652063757272656E74204950204118
:1401F4006464726573730D0A73657469702020202020202056
:140208002020202D20416C6C6F777320796F7520746F2073B0
:14021C006574207468652049502041646464726573730D0A7A
:140230003F75647020202020202020202020202D205072695A
:140244006E7473207468652063757272656E742055445020A4
:14025800416464726573730D0A736574756470202020202080
:14026C00202020202D20416C6C6F777320796F7520746F209F
:14028000736574207468652055445020416464726573730DC1
:140294000A3F75647073656E64706F72742020202D205072E6
:1402A800696E7473207468652063757272656E7420554450F7
:1402BC002053656E6420506F72740D0A73657475647073653B
:1402D0006E64706F7274202D20416C6C6F777320796F752007
:1402E400746F2073657420746865205544502053656E642083
:1402F800506F72740D0A3F75647072656376706F72742020F9
:14030C00202D205072696E7473207468652063757272656EE0
:140320007420554450205265636569766520506F72740D0A8D
:1403340073657475647072656376706F7274202D20416C6C25
:140348006F777320796F7520746F2073657420746865205586
:14035C004450205265636569766520506F72740D0A3F67771D
:140370002020202020202020202020202D205072696E74732C
:14038400207468652063757272656E742047617465776179EF
:1403980020416464726573730D0A736574677720202020208A
:1403AC0020202020202D20416C6C6F777320796F7520746F5E
:1403C000207365742074686520476174657761792041646441
:1403D400726573730D0A3F7375622020202020202020202078
:1403E800202D205072696E7473207468652063757272656E04
:1403FC0074205375624E6574204D61736B0D0A736574737511
:14041000622020202020202020202D20416C6C6F77732079FE
:140424006F7520746F2073657420746865205375624E65749F
:14043800204D61736B0D0A7365746D61696C697020202020A5
:14044C0020202D20416C6C6F777320796F7520746F20736525
:14046000742074686520454D61696C20495020416464726512
:1404740073730D0A3F6D61696C697020202020202020202D8F
:14048800205072696E7473207468652063757272656E74201C
:14049C00454D61696C20495020416464726573730D0A7365F6
:1404B000746D61696C686F7374202020202D20416C6C6F7797
:1404C4007320796F7520746F207365742074686520456D6131
:1404D800696C20486F7374204E616D650D0A3F6D61696C687B
:1404EC006F73742020202020202D205072696E74732074681D
:14050000652063757272656E7420454D61696C20486F7374B9
:14051400204E616D650D0A7365746D61696C73656E646572AB
:1405280020202D20416C6C6F777320796F7520746F20736548
:14053C00742074686520456D61696C2053656E646572204EDF
:14055000616D650D0A3F6D61696C686F7374202020202020ED
:140564002D205072696E7473207468652063757272656E7432
:1405780020454D61696C2053656E646572204E616D650D0A4E
:14058C0073657474696D6520202020202020202D20416C6CFA
:1405A0006F777320796F7520746F207365742074686520631E
:1405B400757272656E742054696D650D0A3F74696D6520209F
:1405C80020202020202020202D205072696E747320746865F1
:1405DC002063757272656E742054696D650D0A736574646111
:1405F000746520202020202020202D20416C6C6F77732079C6
:140604006F7520746F20736574207468652063757272656E7F
:140618007420446174650D0A3F6461746520202020202020E8
:14062C002020202D205072696E747320746865206375727250
:14064000656E7420446174650D0A7365747363686564756C76
:1406540065202020202D20416C6C6F777320796F7520746F6E
:140668002073657420746865205363686564756C6520666975
:14067C006C6520746F206C6F61640D0A3F7363686564756C98
:14069000652020202020202D205072696E74732074686520E3
:1406A40063757272656E74205363686564756C652066696C97
:1406B800650D0A7365746C61746974756465202020202D203D
:1406CC00416C6C6F777320796F7520746F20736574207468C0
:1406E00065204C617469747564650D0A3F6C617469747564F8
:1406F400652020202020202D205072696E747320746865207F
:1407080063757272656E74204C617469747564650D0A73658F
:14071C00746C6F6E6769747564652020202D20416C6C6F77DE
:140730007320796F7520746F2073657420746865204C6F6EAC
:140744006769747564650D0A3F6C6F6E6769747564652020BE
:140758002020202D205072696E747320746865206375727223
:14076C00656E74204C6F6E6769747564650D0A736574746927
:140780006D657A6F6E65202020202D20416C6C6F77732079FF
:140794006F7520746F20736574207468652054696D65205A74
:1407A8006F6E650D0A3F74696D657A6F6E652020202020207A
:1407BC002D205072696E7473207468652063757272656E74D8
:1407D0002054696D65205A6F6E650D0A7365746473742020BC
:1407E400202020202020202D20416C6C6F777320796F7520C5
:1407F800746F2073657420746865204461796C6967687420C7
:14080C00536176696E67732054696D65206D6F64650D0A3F33
:1408200064737420202020202020202020202D204461796C42
:140834006967687420536176696E67732054696D65206D6F5E
:1408480064650D0A3F6572726F727320202020202020202DB3
:14085C00204C6973747320746865206C6173742038206572D5
:14087000726F72732064657465637465640D0A3F5620202040
:14088400202020202020202020202D205072696E74732074BF
:1408980068652063757272656E7420736F66747761726520B1
:1408AC007265766973696F6E00000000000000000047000082
:1408C00000003232302D57656C636F6D6520746F2054686553
:1408D40020416C636F726E204D63427269646520574542736A
:1408E8007465722E0D0A32323020506C65617365206C6F67FC
:1408FC0020696E2E0D0A00343231204D6178696D756D207582
:140910007365727320697320312E0D0A0033333120506173A9
:1409240073776F726420726571756972656420666F72200088
:140938003233302055736572204C6F6767656420696E2E0DB3
:14094C000A00353330204C6F67696E20696E636F7272656367
:14096000742E0D0A0032323120476F6F6462796520616E64F9
:1409740020486176652041204E69636520446179210D0A0055
:1409880032303020547970652073657420746F20492E0D0AEA
:14099C000032303020547970652073657420746F20412E0DE8
:1409B0000A0035303020636F6D6D616E64206E6F7420756E21
:1409C40064657273746F6F642E0D0A0032303020504F52547F
:1409D80020636F6D6D616E64207375636365737366756C2E7E
:1409EC000D0A0032353720222F222069732063757272656E04
:140A000074206469726563746F72792E0D0A0031353020413D
:140A140053434949206461746120636F6E6E656374696F6E9C
:140A28002E0D0A003135302042696E61727920646174612080
:140A3C00636F6E6E656374696F6E2E0D0A0034323520556EB3
:140A500061626C6520746F206F70656E206461746120636F7D
:140A64006E6E656374696F6E2E0D0A0035303020556E6162A0
:140A78006C6520746F2072656164206469726563746F7279E5
:140A8C002E0D0A0035303020556E61626C6520746F206F7003
:140AA000656E2066696C652E0D0A0032353020436F6D6D61C6
:140AB4006E64207375636365737366756C2E0D0A003335301F
:140AC80020436F6D6D616E64207375636365737366756C20BB
:140ADC0070656E64696E67206675727468657220696E666F35
:140AF000726D6174696F6E2E0D0A00323236205472616E73F1
:140B040066657220636F6D706C6574652E0D0A0048545450A2
:140B18002F312E3020323030204F4B0D0A00485454502F31E8
:140B2C002E30203430302042616420526571756573740D0A5C
:140B400000485454502F312E302034303320466F7262696476
:140B540064656E0D0A00485454502F312E3020343034204E1B
:140B68006F7420466F756E640D0A00485454502F312E302045
:140B7C0035303020496E7465726E616C2053657276657220BC
:140B90004572726F720D0A00485454502F312E30203530317C
:140BA400204E6F7420496D706C656D656E7465640D0A0048F9
:140BB8005454502F312E3020353033205365727669636520AA
:140BCC00556E617661696C61626C650D0A0053657276657223
:140BE0003A20416C636F726E204D6342726964652057454294
:140BF400737465720D0A00436F6E74656E742D4C656E677416
:140C0800683A2000436F6E74656E742D547970653A2000749E
:140C1C006578742F68746D6C0D0A00746578742F706C6169DE
:140C30006E0D0A00696D6167652F6A7065670D0A00696D6105
:140C440067652F6769660D0A00696D6167652F706E670D0AC6
:140C5800000D0A0D0A003C48544D4C3E0D0A3C484541443E08
:140C6C000D0A3C5449544C453E003C2F5449544C453E0D0A1F
:140C80003C2F484541443E0D0A3C424F44593E0D0A003C2F64
:140C9400424F44593E0D0A3C2F48544D4C3E0D0A0034303040
:140CA8002042616420526571756573740034303320466F722A
:140CBC0062696464656E00343034204E6F7420466F756E64B9
:140CD0000035303020496E7465726E616C2053657276657287
:140CE400204572726F7200353031204E6F7420496D706C65D4
:140CF8006D656E74656400353033205365727669636520556D
:140D0C006E617661696C61626C65003C48313E3430302048D5
:140D20005454502076657273696F6E206E6F74207375707048
:140D34006F727465643C2F483E003C48313E34303320466F3D
:140D48007262696464656E3C2F483E003C48313E3430342023
:140D5C0046696C65204E6F7420466F756E643C2F483E003C69
:140D700048313E35303020496E7465726E616C2073657276E6
:140D84006572206572726F722C20627566666572206F76650A
:140D980072666C6F772E3C2F483E003C48313E353031204D08
:140DAC006574686F64206E6F7420696D706C656D656E74655E
:140DC000643C2F483E003C48313E3530332046696C65204E31
:140DD4006F7420417661696C61626C652C20747279206167F4
:140DE80061696E206C617465723C2F483E000D0A000D0A2E3A
:140DFC000D0A0046726F6D3A2000546F3A20005375626A65C8
:140E100063743A200048454C4F20004D41494C2046524F4DDE
:140E24003A005243505420544F3A00444154410D0A00515573
:140E380049540D0A004356657273696F6E20423031380000CE
:140E4C0000B4420000704117B7D1380000F040000040410063
:140E600000B44495BFD6341283BB4100003443000070420A64
:140E7400D7A33CB81EF53F4D507C3F96C3B24363537C3F0291
:140E88003B8C430000C0400000803F58FF7F3F000000000078
:140E9C000000400000003F0000C041385A32492A000000008B
:140EB00000000000470000803F0000E8400000B642000035D3
:140EC40043000000470000803F0000E8400000000000202069
:140ED800202020202020203030303030202020202020202036
:140EEC002020202020202020202090404040404040404040E2
:140F00004040404040400C0C0C0C0C0C0C0C0C0C40404040E5
:140F14004040400909090909090101010101010101010101C8
:140F28000101010101010101014040404040400A0A0A0A0AFA
:140F3C000A0202020202020202020202020202020202020271
:140F500002404040402000000000000000000000000000006B
:140F6400000000000000000000000000000000000000000079
:140F7800000000000000000000000000000000000000000065
:140F8C00000000000000000000000000000000000000000051
:140FA00000000000000000000000000000000000000000003D
:140FB400000000000000000000000000000000000000000029
:140FC8000000000000000000000000000000020000007F0094
:140FDC00000000008000FF000000FFFF7F0001000000000004
:140FF00000000000F87FDA0FC93FDB0FC93FE15D25BF5834E5
:14100400A33D632699BBBAD71E39DA0F4940DA0FC93FE4CB21
:141018009640DA0FC9BFDA0FC94082FE7F3FA04DAABE423086
:14102C00463E5B74EEBD02AB573D470A40BCDA0F493F0000B3
:14104000803F00000000DA0F49C0DA0F4940DA0FC9BFDA0F1F
:14105400C93F00000000D10FC93F21A95BBE7FF8B33DCF2659
:1410680038BDC3839E3CD8238EBBDA0FC93F0000803F00006B
:14107C000000FFFFFF7F000000000080FFFFFF7F0000008068
:1410900000000000FFFFFFFF00000000000000000025642E99
:1410A4000025782E002578002564003F45005052494E5453E3
:1410B80043484544554C45000D0A53756E7365743A202530E2
:1410CC00643A2530642E003F53554E534554000D0A53756E1D
:1410E000726973653A202530643A2530642E003F53554E528E
:1410F400495345000D0A4461796C6967687420536176696E99
:1411080067732054696D652069733A20003F445354004F6615
:14111C0066000D0A4461796C6967687420536176696E677311
:141130002054696D65206973206E6F773A20007574005554A0
:14114400007573005553000D0A506C6561736520656E7465CA
:14115800722055532C2055542C206F72206A7573742070723F
:14116C0065737320656E74657220666F72204E4F4E453A00F5
:14118000534554445354000D0A54696D65205A6F6E653A20C8
:14119400474D5420706C75732025306420686F7572732E0023
:1411A8003F54494D455A4F4E45000D0A54696D65205A6F6E8C
:1411BC0065206973206E6F773A20474D5420706C75732025DF
:1411D000306420686F7572732E000D0A506C65617365206502
:1411E4006E7465722054696D65205A6F6E6520696E20686FE5
:1411F80075727328706F736974697665206966206168656150
:14120C0064206F6620474D542C206E65676174697665206945
:141220006620626568696E64293A200053455454494D455AD2
:141234004F4E45003F4C4F4E47495455444500576573740037
:1412480045617374000D0A4C6F6E6769747564653A20253094
:14125C0064202573000D0A506C6561736520656E7465722093
:141270004C6F6E676974756465203020746F203138300D0A9C
:14128400466F726D6174733A0D0A466F7220456173742075C0
:14129800736520655858580D0A466F722057657374207573D4
:1412AC006520775858583A005345544C4F4E47495455444559
:1412C000000D0A4C617469747564653A2025306420257300FC
:1412D4003F4C41544954554445004E6F72746800536F7574B5
:1412E80068000D0A4C61746974756465206973206E6F773A8D
:1412FC0020253064202573000D0A506C6561736520656E7475
:141310006572204C61746974756465203020746F2039300DAD
:141324000A466F726D6174733A0D0A466F72204E6F7274682C
:1413380020757365206E5858580D0A466F7220536F7574682D
:14134C002075736520735858583A005345544C41544954558C
:141360004445003F424F4F54555044454C4159000D0A426FA1
:141374006F742075702064656C61793A2025306420736563E0
:14138800000D0A506C6561736520656E746572206E756D62D0
:14139C006572206F66207365636F6E647320666F7220626F0A
:1413B0006F7475702064656C61793A2000534554424F4F54B8
:1413C400555044454C4159000D0A5363686564756C65206637
:1413D800696C653A202573003F5343484544554C45000D0A32
:1413EC005468652063757272656E74205363686564756C655C
:141400002066696C65206973202573000D0A506C65617365F3
:1414140020656E746572205363686564756C65206E616D6578
:141428002028444F532031312E3320666F726D6174293A2073
:14143C00005345545343484544554C45004356657273696FA8
:141450006E2042303138000D0A56657273696F6E202573204A
:14146400003F560025730D0A2C506C65617365207265636FE1
:141478006E66696775726520796F75722073657269616C20C1
:14148C007465726D696E616C2070726F6772616D2E2E2E004E
:1414A00025730D0A2C53657269616C20666F726D61742077BD
:1414B400696C6C206E6F77206265206368616E6765642E0070
:1414C8000D0A32203D20322073746F702062697473000D0A49
:1414DC0031203D20312073746F7020626974000D0A506C65A0
:1414F0006173652063686F6F7365206E6F2E206F66207374E7
:141504006F7020626974733A000D0A38203D20382062697485
:14151800732F63686172000D0A37203D203720626974732F7C
:14152C0063686172000D0A36203D203620626974732F636841
:141540006172000D0A35203D203520626974732F6368617227
:14155400000D0A506C656173652063686F6F73652062697412
:14156800732F636861723A0033000D0A33203D204576656E6D
:14157C0020506172697479000D0A32203D204F646420506114
:1415900072697479000D0A31203D204E6F2050617269747964
:1415A400000D0A506C656173652063686F6F736520706172BE
:1415B8006974793A00313200313100313000390038003700C1
:1415CC00360035003400320031000D0A0D0A000D0A31322041
:1415E0002D203530304B000D0A3131202D203235304B000DF5
:1415F4000A3130202D203131352E324B000D0A39202D2037D5
:14160800362E384B000D0A38202D2035372E364B000D0A37C2
:14161C00202D2033382E344B000D0A36202D2032382E384B60
:14163000000D0A35202D2031392E324B000D0A34202D2031EF
:14164400342E344B000D0A33202D2039363030000D0A3220C2
:141658002D2034383030000D0A31202D2032343030000D0AD3
:14166C00506C656173652063686F6F73652062617564207221
:141680006174653A0053455453455249414C000D0A437572F5
:1416940072656E74204461746520253032642F253032642F97
:1416A8002530326420000D0A506C6561736520656E74657274
:1416BC002063757272656E74206461746520696E20666F72DB
:1416D0006D204D4D2F44442F5959200053455444415445001D
:1416E4000D43757272656E74204461746520253032642F2505
:1416F8003032642F2530326420003F44415445000D0A4375B2
:14170C007272656E742054696D6520253032643A25303264BF
:141720003A2530326420000D0A506C6561736520656E746533
:14173400722063757272656E742074696D6520696E20666F51
:14174800726D2048523A4D4E3A5353200053455454494D4504
:14175C00000D43757272656E742054696D6520253032643A95
:14177000253032643A2530326420003F54494D45000D0A5060
:141784006C6561736520656E74657220496E697469616C20FF
:14179800574542205061676520696E20666F726D20585858CF
:1417AC0058585858582E48544D293A200053455450414745CE
:1417C000000D0A5468652063757272656E7420496E6974699D
:1417D400616C205745422050616765206973202573003F5056
:1417E800414745003F435553545553455250415353000D0A15
:1417FC0025730D0A25730D0A003F555345525041535300487E
:14181000454C50000D0A4D6564696120686173206265656ED6
:1418240020666F726D61747465642100464F524D4154000DD3
:141838000A5468652063757272656E7420437573746F6D654E
:14184C007220557365726E616D65206973202573000D0A509B
:141860006C6561736520656E74657220437573746F6D6572BA
:1418740020557365726E616D652028313020636861722E204B
:141888006D6178293A200053455443555354005345544355D4
:14189C00535450415353000D0A5468652063757272656E74FF
:1418B00020557365726E616D65206973202573000D0A506C3D
:1418C4006561736520656E74657220557365726E616D6520B4
:1418D80028313020636861722E206D6178293A2000534554B2
:1418EC0055534552000D0A5468652063757272656E742050DE
:14190000617373776F7264206973202573000D0A506C656183
:14191400736520656E7465722050617373776F7264202831BD
:141928003020636861722E206D6178293A2000534554504129
:14193C005353000D0A536F7272792E20204E6F204155544F37
:14195000455845432E4241542066696C6520666F756E64213C
:14196400000D0A416C6C20706172616D6574657273207375E3
:14197800636365737366756C6C7920636F6E6669677572653C
:14198C006421004155544F45584543003F4552524F52530048
:1419A0000D0A506C6561736520656E74657220456D61696C7C
:1419B4002053656E646572204E616D652028692E652E2073F8
:1419C800686F7740726964652E636F6D293A20005345544DB0
:1419DC0041494C53454E444552000D0A54686520637572724C
:1419F000656E7420456D61696C2053656E64657220697320F7
:141A04002573003F4D41494C53454E444552000D0A506C65DB
:141A180061736520656E74657220456D61696C20486F73747D
:141A2C00204E616D652028692E652E20686F73742E636F6D48
:141A4000293A20005345544D41494C484F5354000D0A5468EF
:141A5400652063757272656E7420456D61696C20486F737430
:141A6800206973202573003F4D41494C484F5354000D0A50AF
:141A7C006C6561736520656E74657220456D61696C2049504D
:141A9000204164647265737320696E20666F726D2058585869
:141AA4002E5858582E5858582E5858583A20005345544D41B8
:141AB800494C4950000D0A5468652063757272656E7420452C
:141ACC006D61696C20495020416464726573732069732000A8
:141AE0003F4D41494C4950000D0A506C6561736520656E741F
:141AF4006572205375624E6574204D61736B20696E20666FFE
:141B0800726D205858582E5858582E5858582E5858583A20C6
:141B1C0000534554535542000D0A5468652063757272656EF8
:141B300074205375624E6574204D61736B20697320003F5362
:141B44005542000D0A506C6561736520656E7465722055448E
:141B580050205265636569766520506F7274204E756D62656A
:141B6C00723A200053455455445052454356504F5254000D42
:141B80000A5468652063757272656E742055445020526563C0
:141B94006569766520506F7274206973202575003F554450F1
:141BA80052454356504F5254000D0A506C6561736520656E50
:141BBC00746572205544502053656E6420506F7274204E756F
:141BD0006D6265723A200053455455445053454E44504F5211
:141BE40054000D0A5468652063757272656E74205544502015
:141BF80053656E6420506F7274206973202575003F554450AC
:141C0C0053454E44504F5254000D0A506C6561736520656EF1
:141C200074657220554450204164647265737320696E2066F9
:141C34006F726D205858582E5858582E5858582E5858583A4A
:141C48002000534554554450000D0A5468652063757272651A
:141C5C006E7420554450204164647265737320697320003F48
:141C7000554450000D0A506C6561736520656E746572204761
:141C8400617465776179204164647265737320696E20666FEF
:141C9800726D205858582E5858582E5858582E5858583A2035
:141CAC00005345544757000D0A5468652063757272656E743F
:141CC00020476174657761792041646472657373206973201C
:141CD400003F4757000D0A506C6561736520656E7465722050
:141CE8004D414320494420696E20666F726D2058582E5858F1
:141CFC002E58582E58582E58582E58583A20005345544D4188
:141D100043000D0A5468652063757272656E74204D41432010
:141D2400494420697320003F4D4143000D0A506C6561736581
:141D380020656E746572204950204164647265737320696EC3
:141D4C0020666F726D205858582E5858582E5858582E58583D
:141D6000583A20005345544950000D0A546865206375727224
:141D7400656E74204950204164647265737320697320003F1A
:141D8800495000203D0D0A09003D2009005D006175746F6550
:141D9C007865632E6261740054696D655A6F6E6500004C61B6
:141DB00074697475646500004C6F6E676974756465000042A3
:141DC4006F6F74557044656C617900005363686564756C65D8
:141DD8000000557365726E616D65000050617373776F726464
:141DEC00000046545000005355424D534B31005355424D5369
:141E00004B300047574950310047574950300047617465778C
:141E1400617900004950310049503000310044484350006D90
:141E280061696C6C703100006D61696C6C70300000686F736A
:141E3C0074000073656E6465720000534D545000004D414388
:141E500032004D414331002578004D41433000537973746594
:141E64006D00007363686564756C652E74787400006C6F67E0
:141E7800696E61646D2E68746D0000637573746F6D65720064
:141E8C000061646D696E0000574542737465722E636F6D0030
:141EA00000574542737465724073686F772E636F6D00000024
:141EB4000A0D000D0A000D0A4C6173742038206572726F729F
:141EC800733A00256400000000000000002D2D2D2D2D2D2D95
:141EDC002D2D2D203120657773206577732020202025732004
:141EF000204A616E2020312031303A31322025732E25732078
:141F04000D0A0000467265652073706163653A2025730D0AFB
:141F18000025732E25730D0A0000200D0A002E00524E544F98
:141F2C0000524E46520044454C450053544F52002E00524542
:141F40005452004E4C5354004C49535400505744002C005003
:141F54004F5254005459504500515549540050415353002E9A
:141F68000D0A005553455200200D0A00706E67006A70670052
:141F7C006769660068746D0025640000436F6E74656E742D41
:141F90004C656E6774683A20256400436F6E74656E742D4CA4
:141FA400656E6774683A00436F6E74656E742D6C656E6774B7
:141FB800683A20256400436F6E74656E742D6C656E67746840
:141FCC003A00504F53542000200D0A002E00747874007265C5
:141FE00073756C74732E766172002F726573756C74732E7656
:141FF400617200002F6175746F657865632E62617400002FE5
:14200800257300002F0000485454502F312E310048545450BE
:14201C002F312E3000485454502F302E39000D0A00474554F5
:1420300020002000000A000100010000047363686564756C64
:14204400652E6F6C64007363686564756C652E6E6F77006C7B
:142058006F61642E64617400253032642D253032642D253054
:14206C0032642020253033643A253032643A253032643A25F5
:142080003032640D20000A0D5554204461796C6967687453F0
:142094006176696E677354696D65204F6666000A0D55532007
:1420A8004461796C69676874536176696E677354696D652064
:1420BC004F6666000A0D5554204461796C69676874536176B5
:1420D000696E677354696D65204F6E000A0D555320446179E2
:1420E4006C69676874536176696E677354696D65204F6E0089
:1420F80061646D696E00002B0031323A30303A3030002000E9
:14210C002530640D0020434845434B45440D00200D000D00AB
:14212000726573756C74732E76617200726573756C743D0046
:14213400726573756C74732E747874006E6F6E65006F66660C
:14214800006F6E00736574766172004E414B2052656365692F
:14215C00766564210041434B20526563656976656421007365
:142170007461727473657161636B00436F6D6D616E642053F6
:14218400656E74007374617274736571004E6F205265737012
:142198006F6E736500556E65787065637465642052657370AF
:1421AC006F6E73653A20003C2A00250073656E647374726919
:1421C0006E67006C6F676F7574002A2A2A0025640025730DF0
:1421D4000055540055530075706461746573657474696E6725
:1421E800730073657474696D6500253032643A253032643A2B
:1421FC00253032640D0073657474696E67732E73796E006C72
:142210006F67696E61646D696E00696E64657800766172762D
:14222400616C756500766172696E6465780070617269747905
:142238000073746F706269747300646174616269747300626C
:14224C006175640074797065647465787400646973707265D2
:1422600073756C7400726573706F6E7365737472696E67009C
:14227400737472696E6700617070656E64310073796E6669ED
:142288006C65006E616D65006661696C75726566696C650048
:14229C007375636365737366696C650074696D657A6F6E652A
:1422B000006C61746974756465006C6F6E67697475646500F3
:1422C400626F6F74757064656C6179007363686564756C6511
:1422D80066696C650061646D696E70617373776F7264006175
:1422EC00646D696E757365726E616D650070617373776F72C7
:142300006400757365726E616D650072657175697265757320
:1423140065726C6F67696E00696E697469616C70616765003E
:142328007365727665726970616464726573733400736572CD
:14233C007665726970616464726573733300736572766572B7
:142350006970616464726573733200736572766572697061B7
:142364006464726573733100656D61696C686F737400736511
:142378006E646572656D61696C616464726573730073756270
:14238C006E65746D61736B34007375626E65746D61736B33A6
:1423A000007375626E65746D61736B32007375626E65746DBC
:1423B40061736B310067617465776179616464726573733499
:1423C8000067617465776179616464726573733300676174BA
:1423DC0065776179616464726573733200676174657761792D
:1423F0006164647265737331006970616464726573733400CF
:14240400697061646472657373330069706164647265737313
:1424180032006970616464726573733100656E61626C6564C3
:14242C0068637000656E61626C6573657269616C706F7274B5
:14244000636C6F636B007365636F6E6473006D696E757465FB
:142454007300686F757273007965617200646179006D6F6E97
:142468007468006473740074696D65666F726D00666F726D22
:14247C000026003D00000032323100353534003335340035E5
:14249000353300353531003535300035303300343530003238
:1424A40035310035353200343532003435310035303400351F
:1424B80030310035303000323530003432310032323000B0A8
:1424CC000400000000574542535445522000257300202020C4
:1424E000002020202020202000D00F494014AE073F11111165
:1424F4003F253032643A253032690001000000000000354307
:142508000000B6420F20413A253032642F253032642F253094
:14251C0032640020493A253032643A253032640020523A2591
:14253000306420503A25306420533A2530640020343A257314
:142544000020333A25730020323A25730020313A25730020F7
:14255800453A2530640020443A253032642F253032642F2540
:14256C00303264000D0A543A253032643A253032640053632A
:14258000686564756C65205761726E696E673A2025306400C7
:1425940025732000205363686564756C65204572726F723ACA
:1425A80020253064000D0A0044454641554C545745425041BB
:1425BC004745004F4646004F4E00534554564152455100504C
:1425D000415553450052455345540053544F500053544152C6
:1425E4005453455155454E43450053454E44535452494E4735
:1425F8000000000000FFFF444543004E4F56004F43540053D9
:14260C00455000415547004A554C004A554E004D4159004148
:142620005052004D415200464542004A414E00594541004857
:142634004F55004D494E0053415400465249005448550057F9
:14264800454400545545004D4F4E0053554E004441590053F6
:14265C00554E530053554E5200424F4F00426567616E2050FF
:14267000617273696E673A003C696E7465676572206F6E6C05
:1426840079207072696E742C20757365202D6C66703F3F20B6
:14269800746F2072656C696E6B3E00286E756C6C207074720F
:1426AC0020706173736564290017270061626364656600308E
:1426C000000100616263646566003000756E737570706F72F4
:1426D40074656420666F726D617400617373657274696F6E34
:1426E800206572726F723A2022257322206F6E2066696C65A1
:0D26FC00202573206C696E652025640A009E
:14270A0000E810E010FF006405BFCFEFD0E1CDBFDEBFC456FA
:14271E00D0400AEA08830024E9E6F7E211E8E93CF10711F035
:142732000192FBCF0083E0EAF0E1A0E0B1E117E2E930F107FC
:1427460021F0C89531960D92F9CF0E944856FFCF0E9400E053
:14275A0024978BE899E36C0181E999E35C011601C1010296A0
:14276E006C01F101808191818130E0E09E0709F08DC0160172
:14278200C10102966C01F101808191818030E8E09E0709F061
:1427960081C01601C10102966C01F101808191818430E6E091
:1427AA009E0709F075C01601C10102966C01F1018081918165
:1427BE008130E0E09E0709F069C083EA99E36C011C010296C4
:1427D2006C0140900A3050900B30F1012080318024143504AD
:1427E60009F058C01C0102966C0140900C3050900D30F10191
:1427FA00208031802414350409F04AC08DE999E36C01150191
:14280E00C10102965C0182E090E0F1018083918365E01601C8
:14282200C10102966C012501C20102965C01F2014080518079
:14283600F10140825182862F8150682F882369F783E999E3F7
:14284A006C0144E050E365E01601C10102966C012A014E5FBB
:14285E005F4FF20140805180F10140825182862F8150682F90
:14287200882371F72090A5393090A6392A823B822090A3391D
:142886003090A4392882398226E038E00CE110E00E948C32E1
:14289A0024960E940EE008950E9404E06901780124978BE8AC
:1428AE0099E35C011C0102965C0181E090E0F1018083918351
:1428C2001501C10102965C0180E098E0F1018083918315013E
:1428D600C10102965C0184E096E0F101808391831501C1017C
:1428EA0002965C0181E090E0F1018083918345E064E070E34F
:1428FE001501C10102965C012B016E5F7F4FF20140805180AE
:14291200F10140825182842F8150482F882371F71501C10144
:1429260002965C0144245524F101408251821C0102965C012E
:14293A00F101408251821C0102965C01F101408251821C014C
:14294E0002965C01F101E082F1821C0102965C01F101C08273
:14296200D1828FEF9FEF8A839B838883998326E038E00CE1A5
:1429760010E00E948C3224960E9411E008950E94E1DF0E940F
:14298A008473002309F466C0809169278F3F41F42224209260
:14299E00692701E00E942B3200275BC00E94E272402F20905E
:1429B2000011222009F032C00C3F41F481E080930011222488
:1429C60020926927002749C04D3099F0042F0E945A7E402F69
:1429DA00209069273324C10101968093692785E897E2F1017E
:1429EE00E80FF91F4083002734C020906927222011F400273A
:142A02002EC085E897E2E0916927FF27E80FF91F22242082CE
:142A16002092692701E021C04B3F79F485E897E2E0916927CA
:142A2A00FF27E80FF91F40832224209200110E94E0200027CE
:142A3E0010C0209069273324C10101968093692785E897E23B
:142A5200F101E80FF91F4083002701C000270E94E4DF08959B
:142A66000E9404E0EF97A19780917E27813011F00C949B1F56
:142A7A0027EE3DE105E817E20E9485E30030010739F520900F
:142A8E000A3030900B30232C332420927F2780910A30909195
:142AA2000B3090708093802720900C3030900D30232C33249C
:142AB6002092812780910C3090910D309070809382270AEC55
:142ACA001DE10E94CFE504E00E94BB200C94B11F24EC3DE1A5
:142ADE0005E817E20E9485E30030010709F03FC000E91DE1DD
:142AF2000E94CFE50E94CB1F8091802799279070E0917F275F
:142B0600FF27FE2FEE27E070E82BF92BF0930B30E0930A3061
:142B1A008091822799279070E0918127FF27FE2FEE27E0705C
:142B2E00E82BF92BF0930D30E0930C3020910A3030910B3006
:142B420000E012E00E94933120910C3030910D3002E012E088
:142B56000E9493310AEC1DE10E94CFE504E00E94BB200C94BA
:142B6A00B11F2BE83DE105E817E20E9485E300300107B1F588
:142B7E002090043030900530232C332420927F278091043027
:142B9200909105309070809380272090063030900730232CF3
:142BA60033242092812780910630909107309070809382270F
:142BBA002090083030900930232C33242092832780910830DB
:142BCE009091093090708093842702E71DE10E94CFE506E0B8
:142BE2000E9496200C94B11F2BE63DE105E817E20E9485E3F8
:142BF6000030010709F053C009E31DE10E94CFE50E94442041
:142C0A008091802799279070E0917F27FF27FE2FEE27E0706F
:142C1E00E82BF92BF0930530E0930430809182279927907092
:142C3200E0918127FF27FE2FEE27E070E82BF92BF0930730CC
:142C4600E09306308091842799279070E0918327FF27FE2FE7
:142C5A00EE27E070E82BF92BF0930930E0930830209104307E
:142C6E003091053000E112E00E949331209106303091073044
:142C820002E112E00E949331209108303091093004E112E049
:142C96000E94933106E00E9496200C94B11F25E33DE105E803
:142CAA0017E20E9485E30030010739F520900E3030900F30C0
:142CBE00232C332420927F2780910E3090910F309070809342
:142CD20080272090103030901130232C332420928127809145
:142CE60010309091113090708093822703E11DE10E94CFE544
:142CFA0004E00E94BB200C94B11F2DE03DE105E817E20E9442
:142D0E0085E30030010709F03FC004ED1CE10E94CFE50E9433
:142D2200CB1F8091802799279070E0917F27FF27FE2FEE27BC
:142D3600E070E82BF92BF0930F30E0930E3080918227992715
:142D4A009070E0918127FF27FE2FEE27E070E82BF92BF093EA
:142D5E001130E093103020910E3030910F3004E012E00E9406
:142D72009331209110303091113006E012E00E94933103E174
:142D86001DE10E94CFE504E00E94BB200C94B11F2FEC3CE1DC
:142D9A0005E817E20E9485E30030010739F52090123030901D
:142DAE001330232C332420927F278091123090911330907019
:142DC200809380272090143030901530232C3324209281274A
:142DD600809114309091153090708093822701EB1CE10E94E7
:142DEA00CFE504E00E94BB200C94B11F2AEA3CE105E817E239
:142DFE000E9485E30030010709F03FC005E71CE10E94CFE548
:142E12000E94CB1F8091802799279070E0917F27FF27FE2F3E
:142E2600EE27E070E82BF92BF0931330E093123080918227C7
:142E3A0099279070E0918127FF27FE2FEE27E070E82BF92BBC
:142E4E00F0931530E0931430209112303091133000E415E021
:142E62000E949331209114303091153002E415E00E949331BA
:142E760001EB1CE10E94CFE504E00E94BB200C94B11F28E62A
:142E8A003CE105E817E20E9485E30030010751F42091F57490
:142E9E003091F67406E41CE10E94CFE50C94B11F27E33CE121
:142EB20005E817E20E9485E300300107C9F401E11CE10E94A6
:142EC600CFE50E941D201093F6740093F574980104E415E0E6
:142EDA000E9493312091F5743091F67406E41CE10E94CFE5FC
:142EEE000C94B11F24E03CE105E817E20E9485E30030010717
:142F020051F42091F3743091F4740FED1BE10E94CFE50C9447
:142F1600B11F20ED3BE105E817E20E9485E300300107C9F4C9
:142F2A0007EA1BE10E94CFE50E941D201093F4740093F3746C
:142F3E00980106E415E00E9493312091F3743091F4740FED64
:142F52001BE10E94CFE50C94B11F22EA3BE105E817E20E94F9
:142F660085E30030010731F52090163030901730232C3324EE
:142F7A0020927F2780911630909117309070809380272090C2
:142F8E00183030901930232C33242092812780911830909164
:142FA200193090708093822704E81BE10E94CFE504E00E9452
:142FB600BB20D4C72DE73BE105E817E20E9485E30030010739
:142FCA0009F03DC008E41BE10E94CFE5DFD780918027992791
:142FDE009070E0917F27FF27FE2FEE27E070E82BF92BF09356
:142FF2001730E09316308091822799279070E0918127FF2712
:14300600FE2FEE27E070E82BF92BF0931930E09318302091B5
:14301A0016303091173008E012E00E9493312091183030915A
:14302E0019300AE012E00E94933104E81BE10E94CFE504E0E1
:143042000E94BB208DC720E43BE105E817E20E9485E3003069
:14305600010731F52090114730901247232C332420927F2719
:14306A00809111479091124790708093802720900F473090EF
:14307E001047232C33242092812780910F4790911047907008
:14309200809382270DE11BE10E94CFE504E00E94BB205EC7A8
:1430A60023E13BE105E817E20E9485E30030010709F03DC0D8
:1430BA0009ED1AE10E94CFE569D78091802799279070E09192
:1430CE007F27FF27FE2FEE27E070E82BF92BF0931247E0930A
:1430E20011478091822799279070E0918127FF27FE2FEE2787
:1430F600E070E82BF92BF0931047E0930F47209111473091D2
:14310A0012470CE012E00E94933120910F47309110470EE007
:14311E0012E00E9493310DE11BE10E94CFE504E00E94BB20A4
:1431320017C72FEC3AE105E817E20E9485E30030010739F420
:1431460023E137E400EB1AE10E94CFE507C724EA3AE105E836
:14315A0017E20E9485E300300107C9F403E71AE10E94CFE52E
:14316E000E949121A8019A0103E117E40E947CEA23E137E4AF
:1431820000E712E00E94D33123E137E400EB1AE10E94CFE55F
:14319600E5C627E63AE105E817E20E9485E30030010739F4FD
:1431AA0023E637E406E41AE10E94CFE5D5C628E33AE105E804
:1431BE0017E20E9485E300300107C9F400E01AE10E94CFE5D4
:1431D2000E949121A8019A0103E617E40E947CEA23E637E441
:1431E60000E212E00E94D33123E637E406E41AE10E94CFE5FC
:1431FA00B3C628EF39E105E817E20E9485E30030010719F4E2
:14320E000E945632A7C62FEE39E105E817E20E9485E30030BE
:14322200010771F40E946127002329F005EC19E10E94CFE584
:1432360095C60FE919E10E94CFE590C627E939E105E817E27B
:14324A000E9485E300300107C9F40EE619E10E94CFE50E948B
:14325E009121A8019A0107EE16E40E947CEA27EE36E400E060
:1432720014E00E94D33127EE36E401E519E10E94CFE56EC615
:1432860029E439E105E817E20E9485E300300107C9F400E246
:14329A0019E10E94CFE50E949121A8019A010BEF16E40E94A2
:1432AE007CEA2BEF36E400EB13E00E94D3312BEF36E403E0D7
:1432C20019E10E94CFE54CC627EF38E105E817E20E9485E377
:1432D60000300107C9F40EE619E10E94CFE50E949121A801AE
:1432EA009A010FEB16E40E947CEA2FEB36E400E113E00E948F
:1432FE00D3312FEB36E401E519E10E94CFE52AC62FEE38E128
:1433120005E817E20E9485E300300107C1F40DEB18E10E9437
:14332600CFE5FCD7A8019A0103ED16E40E947CEA23ED36E4AC
:14333A0000EC12E00E94D33123ED36E407E918E10E94CFE592
:14334E0009C620E938E105E817E20E9485E30030010739F425
:143362000E94A99F04E718E10E94CFE5F9C52FE638E105E85A
:1433760017E20E9485E30030010711F4F4D5EEC525E638E163
:14338A0005E817E20E9485E30030010759F487EE96E48883C0
:14339E0099832BEF36E40AE518E10E94CFE5DAC52CE438E1C5
:1433B20005E817E20E9485E30030010759F48FEB96E4888393
:1433C600998323ED36E40AE518E10E94CFE5C6C526E438E1C1
:1433DA0005E817E20E9485E30030010739F42AE637E201E27E
:1433EE0018E10E94CFE5B6C529E138E105E817E20E9485E3EE
:1434020000300107C1F401EE17E10E94CFE588D7A8019A01E9
:143416000AE617E20E947CEA2AE637E200E613E00E94D33109
:14342A002AE637E201E218E10E94CFE595C52BED37E105E8BC
:14343E0017E20E9485E30030010701F500E80E944F5B009382
:14345200EB4302E80E944F5B0093EA4304E80E944F5B009377
:14346600E9432090EB4333242A823B822090EA4333242882AA
:14347A003982202F33270DEB17E10E94CFE56CC525EB37E13B
:14348E0005E817E20E9485E30030010789F507E817E10E94FB
:1434A200CFE569D72090812728822091802700917F270E94EF
:1434B600DA5A00E80E944F5B0093EB4302E80E944F5B009310
:1434CA00EA4304E80E944F5B0093E9430E94565A2090EB439A
:1434DE0033242A823B822090EA433324288239822091E943A4
:1434F200332708E617E10E94CFE532C522E637E105E817E233
:143506000E9485E30030010701F50CE80E944F5B0093EC4377
:14351A0008E80E944F5B0093ED4306E80E944F5B0093EF439F
:14352E002090EC4333242A823B82202E33242882398220912F
:14354200ED43332704E417E10E94CFE509C52CE337E105E8D3
:1435560017E20E9485E30030010789F50EE017E10E94CFE56C
:14356A0058D72090812728822091802700917F270E94155B7B
:14357E000CE80E944F5B0093EC4308E80E944F5B0093ED4338
:1435920006E80E944F5B0093EF430E94565A2090EC4333249E
:1435A6002A823B822090EF433324288239822091ED433327CF
:1435BA000FEE16E10E94CFE5CFC425EE36E105E817E20E946E
:1435CE0085E30030010709F05AC10AEC16E10E94CFE50FEBF8
:1435E20016E10E94CFE504EB16E10E94CFE509EA16E10E94C0
:1435F600CFE50DE916E10E94CFE501E916E10E94CFE505E8A6
:14360A0016E10E94CFE509E716E10E94CFE50DE616E10E9496
:14361E00CFE501E616E10E94CFE503E516E10E94CFE507E490
:1436320016E10E94CFE50BE316E10E94CFE506E316E10E947A
:14364600CFE56CD6A80124E336E10E9485E30030010719F464
:14365A008FECE82E6FC022E336E18A010E9485E300300107B3
:14366E0019F487E6E82E64C020E336E18A010E9485E30030B5
:14368200010719F482E2E82E59C02EE236E18A010E9485E3D0
:143696000030010719F489E1E82E4EC02CE236E18A010E94FB
:1436AA0085E30030010719F480E1E82E43C02AE236E18A0137
:1436BE000E9485E30030010719F48CE0E82E38C028E236E10E
:1436D2008A010E9485E30030010719F488E0E82E2DC026E297
:1436E60036E18A010E9485E30030010719F486E0E82E22C081
:1436FA0023E236E18A010E9485E30030010719F483E0E82E4D
:14370E0017C020E236E18A010E9485E30030010719F4EE24CB
:14372200E3940CC02DE136E18A010E9485E30030010711F459
:14373600EE2402C083E3E82E05E016E10E94CFE505EF15E113
:14374A000E94CFE504EE15E10E94CFE502ED15E10E94CFE59C
:14375E0006E316E10E94CFE5DDD5A80120ED35E10E9485E399
:143772000030010711F462E00BC022E336E18A010E9485E348
:143786000030010711F463E001C0662705EB15E10E94CFE525
:14379A0003EA15E10E94CFE501E915E10E94CFE50FE715E1C0
:1437AE000E94CFE50DE615E10E94CFE506E316E10E94CFE53C
:1437C200AFD5A8012EE236E10E9485E30030010711F4AA248A
:1437D60018C02CE236E18A010E9485E30030010719F4AA243A
:1437EA00A3940DC02AE236E18A010E9485E30030010719F4CA
:1437FE0082E0A82E02C083E0A82E0BE415E10E94CFE50AE35C
:1438120015E10E94CFE508E215E10E94CFE506E316E10E949E
:14382600CFE57CD5A80122E336E10E9485E30030010719F475
:14383A00CC24C39401C0CC2400E015E10E94CFE508EC14E16D
:14384E000E94CFE52E2D00E214E00E948231262F01E214E05E
:143862000E9482312A2D02E214E00E9482312C2D03E214E047
:143876000E9482310E2D0E94E071C8822A2D062F0E94FE71D4
:14388A006BC325EC34E105E817E20E9485E30030010739F481
:14389E0022EB34E107EB14E10E94CFE55BC32DE934E105E881
:1438B20017E20E9485E300300107E1F40CE614E10E94CFE5B5
:1438C6002DD5A8018CE090E0888399839A010AED13E40E9415
:1438DA0078E42AED33E404E214E00E94D3312AED33E40AE4B4
:1438EE0014E10E94CFE536C320E434E105E817E20E9485E379
:143902000030010739F42AED33E40CE214E10E94CFE526C3FC
:143916002DE134E105E817E20E9485E300300107D9F409EE8E
:14392A0013E10E94CFE5F8D4A8010E947AE500939A20202F2D
:14393E00332701E314E00E94933120919A20332700ED13E137
:143952000E94CFE5222420929A2002C323EC33E105E817E28B
:143966000E9485E30030010789F401E314E00E94B931B80171
:14397A000F3FEFEF1E0711F4662777279B0100ED13E10E9499
:14398E00CFE5E8C227EB33E105E817E20E9485E30030010779
:1439A20009F079C004E613E10E94CFE5B9D4A8010E94067D50
:1439B600109369250093682530936B2520936A253A932A938D
:1439CA001A930A930AEB18E00E9493EA3A932A931A930A93BF
:1439DE000E9409DFE4F040906A2550906B25209068253090AB
:1439F20069255A924A923A922A920AEB18E00E9493EA3A930A
:143A06002A931A930A930E9417DE0E94A97FB8016050704823
:143A1A000BC020916A2530916B2500916825109169250E944D
:143A2E00A97FB801262F04E314E00E94823140906A255090DF
:143A42006B2520906825309069255A924A923A922A9206EB14
:143A560018E00E9493EA3A932A931A930A930E9409DF1CF4D7
:143A6A0064E473E102C06EE373E16883798320916A2530915D
:143A7E006B2500916825109169250E94A97F98010AE413E112
:143A92000E94CFE565C224E333E105E817E20E9485E3003068
:143AA600010771F540906A2550906B25209068253090692544
:143ABA005A924A923A922A9206EB18E00E9493EA3A932A9316
:143ACE001A930A930E9409DF1CF464E473E102C06EE373E1FD
:143AE2006883798320916A2530916B2500916825109169250B
:143AF6000E94A97F980101E213E10E94CFE52EC224E133E123
:143B0A0005E817E20E9485E30030010709F079C001EC12E16D
:143B1E000E94CFE5FFD3A8010E94067D109365250093642554
:143B320030936725209366253A932A931A930A930AEB18E031
:143B46000E9493EA3A932A931A930A930E9409DFE4F040904A
:143B5A0066255090672520906425309065255A924A923A9249
:143B6E002A920AEB18E00E9493EA3A932A931A930A930E9405
:143B820017DE0E94A97FB801605070480BC020916625309187
:143B9600672500916425109165250E94A97FB801262F03E38C
:143BAA0014E00E9482314090662550906725209064253090FE
:143BBE0065255A924A923A922A9206EB18E00E9493EA3A9344
:143BD2002A931A930A930E9409DF1CF468EA72E102C063EA8A
:143BE60072E16883798320916625309167250091642510914D
:143BFA0065250E94A97F98010DEA12E10E94CFE5ABC128E90D
:143C0E0032E105E817E20E9485E30030010771F540906625A6
:143C22005090672520906425309065255A924A923A922A924F
:143C360006EB18E00E9493EA3A932A931A930A930E9409DF14
:143C4A001CF468EA72E102C063EA72E168837983209166252C
:143C5E003091672500916425109165250E94A97F98010DEA66
:143C720012E10E94CFE574C12CE832E105E817E20E9485E3A9
:143C860000300107C9F40AE312E10E94CFE546D3A8010E949B
:143C9A007AE500936C25202F05E314E00E94823120916C25D1
:143CAE00332727FD309502E112E10E94CFE552C128E032E165
:143CC20005E817E20E9485E30030010751F420916C253327E5
:143CD60027FD309507EE11E10E94CFE53FC120EE31E105E8A7
:143CEA0017E20E9485E30030010709F05FC08FEF8E870BEAEB
:143CFE0011E10E94CFE50ED3A8010E947AE50E8728EA31E126
:143D12008A010E9485E30030010741F025EA31E18A010E9451
:143D260085E30030010731F481E08093D7438093D9431DC02A
:143D3A0022EA31E18A010E9485E30030010741F02FE931E12F
:143D4E008A010E9485E30030010739F481E08093D74382E077
:143D62008093D94306C022242092D7438FEF8093D9432091E8
:143D7600D94306E314E00E9482310EE711E10E94CFE580919D
:143D8A00D943813029F408EA11E10E94CFE5E4C08091D94330
:143D9E00823029F402EA11E10E94CFE5DBC00AE711E10E94EE
:143DB200CFE5D6C025E731E105E817E20E9485E3003001076D
:143DC600D9F408E511E10E94CFE58091D943813029F408EAFA
:143DDA0011E10E94CFE5C0C08091D943823029F402EA11E133
:143DEE000E94CFE5B7C00AE711E10E94CFE5B2C02FE431E124
:143E020005E817E20E9485E30030010709F03AC022242F8696
:143E16002E86CE010F968C879D87CE010E968A879B87009102
:143E2A006C2511270E94797F0E831F83288739874090662524
:143E3E005090672520906425309065252A823B824C825D826B
:143E520040906A2550906B252090682530906925488259825D
:143E6600222D332D01E00E9466AD2F843324288239822E85E1
:143E7A0033270BE311E10E94CFE56EC023E331E105E817E278
:143E8E000E9485E30030010709F03EC022242F862E86CE0169
:143EA2000F968C879D87CE010E968A879B8700916C25112730
:143EB6000E94797F0E831F83288739874090662550906725F5
:143ECA0020906425309065252A823B824C825D8240906A25EC
:143EDE0050906B25209068253090692548825982222D332D81
:143EF20000270E9466AD2F84332427FC3094288239822E85D7
:143F0600332727FD309500E211E10E94CFE526C022E131E13F
:143F1A0005E817E20E9485E30030010719F40E94607D1AC005
:143F2E0001E00E942B3216C02FE031E105E817E20E9485E3B8
:143F42000030010751F40E948332402F242F33270CE011E19D
:143F56000E94CFE503C001E00E942B32EF96A1960E9411E00F
:143F6A0008950E94F8DF6EE471E0442708C01B016F5F7F4F9F
:143F7E00F1014491042F0E9443EAFB01E491EE23A1F70E94AA
:143F920008E008950E94FCDF6297AA24442766270E94A173A4
:143FA6002FC00E948473002359F10E94E272A02E0E9443EA7F
:143FBA008A2D8E32D1F4CE010296E62FFF27E80FF91F2224C0
:143FCE0020828FE797E2242E3324280E391E288239822CE0A7
:143FE20031E18E010E5F1F4F0E946AE64395662709C0262EDB
:143FF60033246F5FCE010296F101E80FF91FA0828A2D8D3094
:14400A0009F0CDCF0A2D0E9443EA8FE797E2242E3324280E39
:14401E00391E288239822CE031E18E010E5F1F4F0E946AE658
:1440320062960E940BE008950E94F8DF2697662744270E9488
:14404600A17311C00E948473002369F00E94E272602F0E9445
:14405A0043EA242E33244F5FCE01F101E80FF91F60836D307E
:14406E0011F0463058F3062F0E9443EA8E010E947AE526962C
:144082000E9408E008950E94FCDF6497AA24442766270E9423
:14409600A1732FC00E948473002359F10E94E272A02E0E94A7
:1440AA0043EA8A2D8E32D1F4CE010296E62FFF27E80FF91FE8
:1440BE00222420828FE797E2242E3324280E391E288239827C
:1440D20029E031E18E010E5F1F4F0E946AE64395662709C035
:1440E600262E33246F5FCE010296F101E80FF91FA0828A2D0C
:1440FA008D3009F0CDCF0A2D0E9443EA8FE797E2242E3324C2
:14410E00280E391E2882398229E031E18E010E5F1F4F0E9484
:144122006AE664960E940BE008950E94F8DF602F44270DC0D5
:144136008FE797E2E42FFF27E80FF91F2081332705E011E16C
:14414A000E94CFE54395862F8250841778F78EE797E2E62F9F
:14415E00FF27E80FF91F2081332709E011E10E94CFE50E944A
:1441720008E008950E94F8DF602F44270DC08FE797E2E42F72
:14418600FF27E80FF91F2081332701E011E10E94CFE54395F4
:14419A00862F8250841778F78EE797E2E62FFF27E80FF91F48
:1441AE00208133270CE011E10E94CFE50E9408E008950E9405
:1441C20004E0EF97EF97EF97EF97259766274427AA2471C03A
:1441D600CE010296C42EDD24C80ED91E0FC085E897E2E42FE6
:1441EA00FF27E80FF91F6081CE010296E42FFF27E80FF91FFC
:1441FE006083439585E897E2E42FFF27E80FF91F20802220E2
:1442120041F7242E33244F5FCE010296F101E80FF91F22245B
:144226002082CE010296E42EFF24E80EF91E0FC085E897E284
:14423A00E42FFF27E80FF91F6081CE010296E42FFF27E80FB0
:14424E00F91F6083439585E897E2E42FFF27E80FF91F2080BB
:14426200222041F7242E33244F5FCE010296F101E80FF91F0F
:1442760022242082CE010296A42EBB24A80EB91E0FC085E86B
:14428A0097E2E42FFF27E80FF91F6081CE010296E42FFF27DE
:14429E00E80FF91F6083439585E897E2E42FFF27E80FF91F14
:1442B20080818B3F41F785E897E2E42FFF27E80FF91F8081C6
:1442C6008B3F09F085CFCE010296E42FFF27E80FF91F2224D8
:1442DA00208280E18093302F2092312FA882B98297018601C5
:1442EE000E94516C002349F480E28093302F8093312F04E0D2
:144302000E942B3205C022242092302F2092312FEF96EF9670
:14431600EF96EF9625960E9411E008950E94FCDFEF976197A3
:14432A00662744270E94A1730E948473002361F00E94E272CE
:14433E00602F0E9443EACE01E42FFF27E80FF91F608343953B
:144352006D3071F74A95CE01E42FFF27E80FF91F2224208274
:14436600CE015C01082F192FEF9661960E940BE008950E9450
:14437A00FCDF2C97AA24442766270E94A1732FC00E9484738D
:14438E00002359F10E94E272A02E0E9443EA8A2D8A33D1F4E2
:1443A200CE010296E62FFF27E80FF91F222420828FE797E27F
:1443B600242E3324280E391E288239822CE031E18E010E5F3E
:1443CA001F4F0E946AE64395662709C0262E33246F5FCE0109
:1443DE000296F101E80FF91FA0828A2D8D3009F0CDCF0A2DD0
:1443F2000E9443EA8FE797E2242E3324280E391E288239825E
:144406002CE031E18E010E5F1F4F0E946AE62C960E940BE0D9
:14441A0008950E94FCDF2C97AA24442766270E94A17331C044
:14442E000E948473002369F10E94E272A02E0E9443EA8A2D1A
:144442008F3211F08E32D1F4CE010296E62FFF27E80FF91F6E
:14445600222420828FE797E2242E3324280E391E28823982E0
:14446A002CE031E18E010E5F1F4F0E946AE64395662709C096
:14447E00262E33246F5FCE010296F101E80FF91FA0828A2D70
:144492008D3009F0CBCF0A2D0E9443EA8FE797E2242E332428
:1444A600280E391E288239822CE031E18E010E5F1F4F0E94E6
:1444BA006AE62C960E940BE008950E9404E06901A80167971B
:1444CE00A9A0BAA0EBA0FCA00E94A173CC2019F4DD2009F467
:1444E2005FC066273BC08A010E94CFE522242A822A2D33279B
:1444F60000E21EE40E94E97E0093E84328C00E948473002363
:14450A0021F12A2D332700E21EE40E94E97E0093E8430E948D
:14451E00E2720E8B81E090E0888399839E012A5E3F4F8E0160
:144532000E5F1F4F0E9432E596018E010E5F1F4F0E9485E3D6
:144546000030010721F422242092E8436E2D2090E843222039
:14455A00A1F663956E1508F4C2CF8E010E5F1F4F0E9426E597
:14456E000030010759F096018E010E5F1F4F0E9485E300307D
:14458200010711F006E910C08E010E5F1F4F0E9426E5003016
:14459600010711F406E906C0002704C08A010E94CFE500275C
:1445AA0067960E9411E008950E94E1DF44272224209285285E
:1445BE0011C04F3F29F4442701E00E942B320EC00E94E2725E
:1445D20086E898E2E42FFF27E80FF91F008343950E948473B1
:1445E600002359F786E898E2E42FFF27E80FF91F2224208236
:1445FA0003D00E94E4DF08950E94E1DF809186288C3F11F4E7
:14460E00F2D018C0809186288F3389F480918728853481F412
:14462200209088282092E7430E948332402F42E0242F00917C
:14463600E74325D003C001E00E942B320E94E4DF08950E940A
:14464A00F8DF602F462F495E21E00FEF0E94F6722227002761
:14465E000E94F672222708E10E94F6722227062F0E94F6727A
:1446720046954F7721E0042F0E94F6720E9408E008950E948C
:14468600FCDF622FA02E4A2D495D460F21E00FEF0E94F6726B
:14469A00222700270E94F672222708E20E94F67222270A2DD5
:1446AE000E94F6722227062F0E94F67246954F7721E0042F91
:1446C2000E94F6720E940BE008950E94F8DF602F462F4F5F85
:1446D60021E00FEF0E94F672222700270E94F672222702E022
:1446EA000E94F6722227062F0E94F67246954F7721E0042F55
:1446FE000E94F67200270E9408E008950E94F8DF602F462FD3
:144712004E5F21E00FEF0E94F672222700270E94F67222271A
:1447260003E00E94F6722227062F0E94F67246954F7721E068
:14473A00042F0E94F67200270E9408E008950E94F8DFB801AE
:14474E00CB019070AB01452F55275070415C480F21E00FEF3C
:144762000E94F672222700270E94F672222700E40E94F67288
:1447760022278B0110700E94F67222278B01012F1127107013
:14478A000E94F67246954F7721E0042F0E94F6720E94AC7371
:14479E000E948473002319F00E94E27201C000270E9408E0DA
:1447B20008950E94FCDFB80114C04427552709C08B010E946E
:1447C6005B38A02E22270E94F6724F5F5F4F4034E0E05E0736
:1447DA0098F306E910E00E94984B8B010E945039002339F3D6
:1447EE000E940BE008950E9404E0EF97EF97EF97EF97259733
:14480200662741E0AA2471C0CE010296C42EDD24C80ED91ECE
:144816000FC086E898E2E42FFF27E80FF91F6081CE01029647
:14482A00E42FFF27E80FF91F6083439586E898E2E42FFF2756
:14483E00E80FF91F2080222041F7242E33244F5FCE0102967F
:14485200F101E80FF91F22242082CE010296E42EFF24E80ED7
:14486600F91E0FC086E898E2E42FFF27E80FF91F6081CE0178
:14487A000296E42FFF27E80FF91F6083439586E898E2E42F94
:14488E00FF27E80FF91F2080222041F7242E33244F5FCE01A1
:1448A2000296F101E80FF91F22242082CE010296A42EBB2469
:1448B600A80EB91E0FC086E898E2E42FFF27E80FF91F608181
:1448CA00CE010296E42FFF27E80FF91F6083439586E898E288
:1448DE00E42FFF27E80FF91F80818B3F41F786E898E2E42F80
:1448F200FF27E80FF91F80818B3F09F085CFCE010296E42FEB
:14490600FF27E80FF91F22242082A882B982970186010E945A
:14491A00516C002349F480E28093302F8093312F04E00E949F
:14492E002B3205C022242092302F2092312FEF96EF96EF965B
:14494200EF9625960E9411E008950E9404E0219700E112E0E0
:144956000E94B931109305300093043002E112E00E94B931C1
:14496A00109307300093063004E112E00E94B9311093093057
:14497E000093083080910430909105308F3FEFEF9E0711F568
:1449920080910630909107308F3FEFEF9E07D1F48091083013
:1449A600909109308F3FEFEF9E0791F480E190E090930530A4
:1449BA008093043080E096E4909307308093063081E797E145
:1449CE0090930930809308302090F143222009F080C000E0EF
:1449E20012E00E94B93110930B3000930A3002E012E00E9422
:1449F600B93110930D3000930C3080910A3090910B308F3F9F
:144A0A00EFEF9E07A1F480910C3090910D308F3FEFEF9E0784
:144A1E0061F488EA90EC90930B3080930A308EEF90E0909386
:144A32000D3080930C3004E012E00E94B93110930F3000930D
:144A46000E3006E012E00E94B93110931130009310308091F2
:144A5A000E3090910F308F3FEFEF9E0791F480911030909162
:144A6E0011308F3FEFEF9E0751F42224332430920F3020920D
:144A82000E30309211302092103008E012E00E94B9311093E4
:144A96001730009316300AE012E00E94B93110931930009305
:144AAA00183080911630909117308F3FEFEF9E0791F480910A
:144ABE001830909119308F3FEFEF9E0751F42224332430923D
:144AD200173020921630309219302092183000E415E00E9411
:144AE600B931109313300093123002E415E00E94B93110930D
:144AFA0015300093143080911230909113308F3FEFEF9E0784
:144B0E0091F480911430909115308F3FEFEF9E0751F4222477
:144B220033243092133020921230309215302092143004E44A
:144B360015E00E94B9311093F6740093F5740F3FEFEF1E0790
:144B4A0031F48FE49AE09093F6748093F57406E415E00E94BB
:144B5E00B9311093F4740093F3740F3FEFEF1E0731F48FE46B
:144B72009AE09093F4748093F37400E212E00E94B931B80197
:144B86000F3FEFEF1E0739F421E03FE103E617E40E947CEA90
:144B9A000AC000E212E00E94F2315801950103E617E40E942F
:144BAE007CEA00E712E00E94B931B8010F3FEFEF1E0739F4F1
:144BC20024EF3EE103E117E40E947CEA0AC000E712E00E9481
:144BD600F2315801950103E117E40E947CEA0CE012E00E9452
:144BEA00B93110931247009311470EE012E00E94B9311093D7
:144BFE00104700930F4780911147909112478F3FEFEF9E072F
:144C120081F40F3FEFEF1E0761F488EA90EC909312478093F6
:144C2600114780EF90E09093104780930F4700E014E00E94EA
:144C3A00B931B8010F3FEFEF1E0739F42DEE3EE107EE16E41C
:144C4E000E947CEA0AC000E014E00E94F2315801950107EE03
:144C620016E40E947CEA00EB13E00E94B931B8010F3FEFEFED
:144C76001E0739F42DEE3EE10BEF16E40E947CEA0AC000EBED
:144C8A0013E00E94F231580195010BEF16E40E947CEA00E192
:144C9E0013E00E94B931B8010F3FEFEF1E0739F423EE3EE11C
:144CB2000FEB16E40E947CEA0AC000E113E00E94F231580136
:144CC60095010FEB16E40E947CEA00EC12E00E94B931B80125
:144CDA000F3FEFEF1E0739F423EE3EE103ED16E40E947CEA26
:144CEE000AC000EC12E00E94F2315801950103ED16E40E94CA
:144D02007CEA00E613E00E94B931B8010F3FEFEF1E0739F49B
:144D160025ED3EE10AE617E20E947CEA0AC000E613E00E9422
:144D2A00F231580195010AE617E20E947CEA00E214E00E94FA
:144D3E00A831402F0F3F21F403E30E94E07103C0042F0E9445
:144D5200E07101E214E00E94A831402F0F3F39F422242882D0
:144D660023E000270E94FE710FC002E214E00E94A831C02EEE
:144D7A0003E214E00E94A831E02EE8822C2D042F0E94FE71BC
:144D8E0004E214E00E94B931B8010F3FEFEF1E0739F427EC61
:144DA2003EE10AED13E40E947CEA0AC004E214E00E94F2317F
:144DB600580195010AED13E40E947CEA01E314E00E94B931A0
:144DCA00B8010F3FEFEF1E0721F4222420929A2002C060934F
:144DDE009A2003E314E00E94A831402F0F3F69F40EEB18E0A7
:144DF2000E9493EA10936525009364253093672520936625B8
:144E06000CC0042F11270E94797F10936525009364253093BB
:144E1A0067252093662504E314E00E94A831402F0F3F69F44A
:144E2E000EEB18E00E9493EA109369250093682530936B25BC
:144E420020936A250CC0042F11270E94797F10936925009385
:144E5600682530936B2520936A2505E314E00E94A831402F60
:144E6A000F3F21F4222420926C2502C040936C2506E314E045
:144E7E000E94A831402F0F3F39F48FEF8093D9432224209216
:144E9200D74305C04093D94381E08093D74307E314E00E9430
:144EA600A831402F0F3F21F422242092D84302C04093D8438A
:144EBA0021960E9411E00895EE97CE010296888399832AEBD5
:144ECE003EE10FEB1EE1AED1002359F084E090E388839983CF
:144EE20027EB3EE18E010E5F1F4F0E946AE6CE0102968883BD
:144EF600998322EB3EE10FEB1EE198D1002359F086E090E3B9
:144F0A008883998327EB3EE18E010E5F1F4F0E946AE6CE0110
:144F1E000296888399832DEA3EE10FEB1EE182D1002359F0D2
:144F320088E090E38883998327EB3EE18E010E5F1F4F0E942C
:144F46006AE683E697E4888399832FE93EE107EA1EE16CD198
:144F5A0083E197E48883998329E93EE107EA1EE163D1CE0119
:144F6E0002968883998320E93EE107EA1EE15AD1002301F415
:144F820081E197E48883998327EB3EE18E010E5F1F4F0E94DA
:144F96006AE6CE0102968883998327E83EE107EA1EE144D1F6
:144FAA00002301F48FE097E48883998327EB3EE18E010E5F9D
:144FBE001F4F0E946AE6CE0102968883998322E83EE10FEBCE
:144FD2001EE12ED10023A9F081E090E08883998320E83EE1F2
:144FE6008E010E5F1F4F0E9435E40030010721F481E08093D1
:144FFA00F14303C022242092F1432090F143222009F0A0C001
:14500E00CE010296888399832CE73EE10FEB1EE109D10023D8
:1450220059F08AE090E38883998327EB3EE18E010E5F1F4F92
:145036000E946AE6CE0102968883998328E73EE10FEB1EE1BF
:14504A00F3D0002359F08CE090E38883998327EB3EE18E015D
:14505E000E5F1F4F0E946AE6CE0102968883998329E63EE1B5
:145072000FE61EE1DDD0002361F08EE090E38883998327EBFB
:145086003EE18E010E5F1F4F0E946AE606C022243324309276
:14509A000F3020920E30CE0102968883998323E63EE10FE628
:1450AE001EE1C0D0002361F080E190E38883998327EB3EE1BF
:1450C2008E010E5F1F4F0E946AE606C0222433243092113018
:1450D60020921030CE010296888399832BE53EE10FE61EE123
:1450EA00A3D0002361F086E190E38883998327EB3EE18E010A
:1450FE000E5F1F4F0E946AE606C08FEF9FEF90931730809382
:145112001630CE0102968883998323E53EE10FE61EE186D044
:14512600002361F088E190E38883998327EB3EE18E010E5FD1
:14513A001F4F0E946AE606C08FEF9FEF909319308093183068
:14514E0087EE96E48883998324E43EE10EE41EE169D08BEF6C
:1451620096E4888399832AE33EE10EE41EE160D08AED93E45D
:145176008883998320E33EE10FEB1EE157D0CE01029688834A
:14518A00998323E23EE10FEB1EE14ED0002339F08E010E5F72
:14519E001F4F0E947AE500939A20CE0102968883998328E1AA
:1451B2003EE10FEB1EE13CD0002369F08E010E5F1F4F0E943D
:1451C600067D10936525009364253093672520936625CE01AD
:1451DA000296888399832EE03EE10FEB1EE124D0002369F06C
:1451EE008E010E5F1F4F0E94067D109369250093682530930A
:145202006B2520936A25CE0102968883998324E03EE10FEB1B
:145216001EE10CD0002339F08E010E5F1F4F0E947AE500935F
:14522A006C2501E0EE9608950E947FDF0E9404E05901E49782
:14523E00FE01EE5BFF4F6081718122E707EF1DE10E945B36C3
:14525200A8010030010709F03DC0002795C082E390E0888315
:1452660099839E012E5F3F4F8A010E940D39E02ECE01029676
:14527A00EE2DFF27E80FF91F222420828A818B3529F525EFEB
:14528E003DE18E010D5F1F4F0E94D6E268010E9426E51801FC
:1452A2000EAD1FAD2F923F920E9426E53F902F902016310637
:1452B60079F40EAD1FAD0E9426E50883198396010EAD1FADFE
:1452CA000E9435E40030010709F450C08A010E9450390023F7
:1452DE0009F4BFCF49C082E390E0888399839E012E5F3F4F72
:1452F2008A010E940D39E02ECE010296EE2DFF27E80FF91F70
:145306002224208221EF3DE18E010E5F1F4F0E94D6E2680150
:14531A008A818B3509F430C086010E9426E5180185012F9233
:14532E003F920E9426E53F902F9020163106E1F485010E94F5
:1453420026E508831983950186010E9435E40030010781F4A0
:145356002BEE3DE1002711270E94D6E2680196018B010E9425
:14536A007CEA8A010E943F3A01E00AC08A010E94503900239F
:14537E0009F4B1CF8A010E943F3A0027E4960E9411E024960A
:1453920008950E9400E006E3A5D68CE99AE2A801480F591F1B
:1453A60005E39ED68CE99AE2F801E80FF91F608182E0A82E85
:1453BA00C090131FDD24CC2011F4DD2029F1C6018130E0E01C
:1453CE009E0709F46BC08230E0E09E0709F4F3C08330E0E0C4
:1453E2009E0709F4FFC08430E0E09E0709F451C18530E0E0B9
:1453F6009E0709F4E6C38630E0E09E0709F458C28730E0E0AF
:14540A009E0709F49FC2D2CF81E080939420002711270E94C1
:14541E00B93110938C2900938B2902E010E00E94B9311093F0
:145432008E2900938D2904E010E00E94B9311093982900930F
:14544600972906E010E00E94B93110939A290093992908E08D
:14545A0010E00E94B93110939429009393290AE010E00E9497
:14546E00B931109396290093952980918B2990918C298F3F24
:14548200EFEF9E0761F480918D2990918E298F3FEFEF9E074E
:1454960021F482E08093131F8BCF65D481E08093131F86CFB8
:1454AA0022E003E00A19E4D3002309F47DC005E315D68CE98A
:1454BE009AE2F801E80FF91F6081653009F06BC006E30AD6F3
:1454D2008AE99AE2A801480F591FFA018381992790703296D8
:1454E600E081FF27FE2FEE27E070E82BF92BF0939029E093B3
:1454FA008F29FA018581992790703496E081FF27FE2FEE2792
:14550E00E070E82BF92BF0939229E093912920908B29309073
:145522008C2930920B3020920A3020908D2930908E29309238
:145536000D3020920C30209093293090942930921730209292
:14554A00163020909529309096293092193020921830209065
:14555E0097293090982930920F3020920E30209099293090D5
:145572009A2930921130209210309F0100918F29109190292A
:145586000E943935FED5222433243092A02920929F292092DA
:14559A00942085E08093131F09CF663009F006CF82E08093EE
:1455AE00131F02CFAA2021F482E08093131FFCCEAA94D5D3B0
:1455C200F9CE81E0809394202224332430920B3020920A3060
:1455D60030920D3020920C3083E08093131FE8CE7ED322E023
:1455EA0002E046D3002309F4E1CEA0D5002309F4DDCE06E3BA
:1455FE0073D58AE99AE2A801480F591FFA018381992790702B
:145612003296E081FF27FE2FEE27E070E82BF92BF093902930
:14562600E0938F29FA018581992790703496E081FF27FE2F06
:14563A00EE27E070E82BF92BF0939229E09391298091BF295C
:14564E0099279070E091BE29FF27FE2FEE27E070E82BF92B41
:14566200F0938C29E0938B298091C12999279070E091C029C0
:14567600FF27FE2FEE27E070E82BF92BF0938E29E0938D29CE
:14568A0070D384E08093131F91CE22E003E00A19EFD20023D5
:14569E0009F401C105E320D58CE99AE2F801E80FF91F608182
:1456B200653009F0EFC03ED5002309F4EBC08091BF29992710
:1456C6009070E091BE29FF27FE2FEE27E070E82BF92BF09306
:1456DA000B30E0930A308091C12999279070E091C029FF2799
:1456EE00FE2FEE27E070E82BF92BF0930D30E0930C302091BF
:145702000A3030910B30002711270E94933120910C303091EA
:145716000D3002E010E00E94933101E0E1D4180101E02F92B9
:14572A003F92DCD43F902F908DE99AE2F801E80FF91F808161
:14573E0099279070ECE9FAE2D101AE0FBF1FEC91FF27FE2FA9
:14575200EE27E070E82BF92BF0931730E093163001E0C0D4AF
:14576600180101E02F923F92BBD43F902F908FE99AE2F80199
:14577A00E80FF91F808199279070EEE9FAE2D101AE0FBF1F2B
:14578E00EC91FF27FE2FEE27E070E82BF92BF0931930E0935C
:1457A2001830209116303091173008E010E00E9493312091BD
:1457B6001830309119300AE010E00E94933103E08FD41801EE
:1457CA0003E02F923F928AD43F902F908DE99AE2F801E80F88
:1457DE00F91F808199279070ECE9FAE2D101AE0FBF1FEC9143
:1457F200FF27FE2FEE27E070E82BF92BF0930F30E0930E3041
:1458060003E06ED4180103E02F923F9269D43F902F908FE998
:14581A009AE2F801E80FF91F808199279070EEE9FAE2D101B0
:14582E00AE0FBF1FEC91FF27FE2FEE27E070E82BF92BF093DC
:145842001130E093103020910E3030910F3004E010E00E94F9
:145856009331209110303091113006E010E00E94933120919A
:14586A0091293091922900918F29109190290E94393585D4E8
:14587E00222433243092A02920929F292092942085E0809396
:14589200131F90CD663009F08DCD82E08093131F89CDAA20C3
:1458A60021F482E08093131F83CDAA945CD280CD2090A329AD
:1458BA00222021F056D222242092A32924EA39E204E410E09A
:1458CE000E94D9750023C9F0653071F42DD4002359F053D46C
:1458E200222433243092A02920929F2985E08093131F09C09D
:1458F600663039F41DD4002321F082E08093131F57CD20903B
:14590A009B2930909C2940909F295090A0294214530408F456
:14591E004BCD910101E010E00E94E97E23E030E00E94B27E0C
:1459320010939C2900939B29222433243092A02920929F2900
:1459460087E08093131F34CD2090A329222021F00AD22224AF
:14595A002092A32924EA39E204E410E00E94D975002309F4AA
:14596E0016C1653009F00AC1DFD3002309F406C18091BF2963
:1459820099279070E091BE29FF27FE2FEE27E070E82BF92B0A
:14599600F0930B30E0930A308091C12999279070E091C0297D
:1459AA00FF27FE2FEE27E070E82BF92BF0930D30E0930C308B
:1459BE0020910A3030910B30002711270E94933120910C303C
:1459D20030910D3002E010E00E94933101E082D3180101E05B
:1459E6002F923F927DD33F902F908DE99AE2F801E80FF91F43
:1459FA00808199279070ECE9FAE2D101AE0FBF1FEC91FF2717
:145A0E00FE2FEE27E070E82BF92BF0931730E093163001E057
:145A220061D3180101E02F923F925CD33F902F908FE99AE2FF
:145A3600F801E80FF91F808199279070EEE9FAE2D101AE0F51
:145A4A00BF1FEC91FF27FE2FEE27E070E82BF92BF093193032
:145A5E00E0931830209116303091173008E010E00E9493313C
:145A720020911830309119300AE010E00E94933103E030D3F7
:145A8600180103E02F923F922BD33F902F908DE99AE2F80107
:145A9A00E80FF91F808199279070ECE9FAE2D101AE0FBF1F0A
:145AAE00EC91FF27FE2FEE27E070E82BF92BF0930F30E09343
:145AC2000E3003E00FD3180103E02F923F920AD33F902F90D4
:145AD6008FE99AE2F801E80FF91F808199279070EEE9FAE24C
:145AEA00D101AE0FBF1FEC91FF27FE2FEE27E070E82BF92BCF
:145AFE00F0931130E093103020910E3030910F3004E010E05A
:145B12000E949331209110303091113006E010E00E949331EA
:145B2600FA018381992790703296E081FF27FE2FEE27E070CB
:145B3A00E82BF92BF0939029E0938F29FA01858199279070F8
:145B4E003496E081FF27FE2FEE27E070E82BF92BF0939229EB
:145B6200E09391299F0100918F29109190290E94393509D3D3
:145B7600222433243092A02920929F2985E08093131F09C006
:145B8A00663039F4D3D2002321F082E08093131F0DCC20903B
:145B9E009B2930909C2940909F295090A0294214530408F4C0
:145BB20001CC222433243092A02920929F2982E08093131FC9
:145BC600F7CB20909B2930909C2940909F295090A029421479
:145BDA005304B8F0910103E010E00E94E97E180136942794AC
:145BEE003694279430929C2920929B29222433243092A029F9
:145C020020929F2986E08093131F0E940EE0089580919D2965
:145C160090919E29019690939E2980939D292090A1293090FE
:145C2A00A229222011F4332039F0222433243092A2292092FC
:145C3E00A12995D08DE194E020909D2930909E298215930515
:145C520090F42224332430929E2920929D2980919F29909122
:145C6600A02901969093A02980939F2981E08093A329089526
:145C7A000E94F8DF422F602F83E0861708F463E08EB58D602E
:145C8E008EBD262F332705E515E50E94E97EC8010197909397
:145CA2004B0080934A0086B7806186BF2224332430924D0037
:145CB60020924C0024EA39E204E410E00E94D975002331F0A7
:145CCA002090AE292416A1F701E004C026B624FEEFCF0027E5
:145CDE000E9408E008950E94E1DF28970E9466E5009387293A
:145CF2000E9466E5009388290E9466E5009389290E9466E54E
:145D060000938A2940D14EE95AE21A014F5F5F4F85E3F101EE
:145D1A0080831A014F5F5F4F81E0F10180831A014F5F5F4F2E
:145D2E00F10180831A014F5F5F4F8FEFF101808383E490E0AB
:145D42008E839F8384E48C839D838FEF9FEF8A839B83888341
:145D5600998324EF30E00EEA19E20E94287528960E94E4DFA5
:145D6A0008950E94F8DF289748E06AEB79E209D18091131F5B
:145D7E00863011F08730F1F480910A3090910B30892F99279F
:145D92009070FB01848780910A3090910B3090708587809132
:145DA6000C3090910D30892F99279070868780910C3090915C
:145DBA000D30907087874C5F6EE97AE21B016F5F7F4F85E30C
:145DCE00F10180831B016F5F7F4F81E0F10180831B016F5FD4
:145DE2007F4F83E0F10180838091131F863009F440C08730DA
:145DF60009F43DC01B016F5F7F4F82E3F10180831B016F5FA3
:145E0A007F4F84E0F10180831B016F5F7F4F80918B299091BF
:145E1E008C29892F992787FD90959070F10180831B016F5FBB
:145E32007F4F80918B2990918C299070F10180831B016F5F14
:145E46007F4F80918D2990918E29892F992787FD90959070BA
:145E5A00F10180831B016F5F7F4F80918D2990918E299070E8
:145E6E00F10180834A5F8091131F833019F0843009F03DC0D9
:145E82001B016F5F7F4F86E3F10180831B016F5F7F4F84E0DA
:145E9600F10180831B016F5F7F4F80918F2990919029892FF0
:145EAA00992787FD90959070F10180831B016F5F7F4F8091BD
:145EBE008F29909190299070F10180831B016F5F7F4F809180
:145ED200912990919229892F992787FD90959070F101808310
:145EE6004A5F1B016F5F7F4F80919129909192299070F101AE
:145EFA0080831B016F5F7F4F8FEFF10180838091131F86306D
:145F0E0029F583E490E08E839F8384E48C839D832090912956
:145F2200309092292A823B8220908F29309090292882398241
:145F3600242F332724513F4F0EEA19E20E942875003001073D
:145F4A00E1F481E090E09093A2298093A12915C083E490E026
:145F5E008E839F8384E48C839D838FEF9FEF8A839B83888323
:145F72009983242F332724513F4F0EEA19E20E94287528965F
:145F86000E9408E008950EEA19E22EEA39E281E091E0F801EF
:145F9A008083918386E090E08283938380918729992790706A
:145FAE00E0918829FF27FE2FEE27E070E82BF92BD80114964B
:145FC200ED93FC938091892999279070E0918A29FF27FE2FC2
:145FD600EE27E070E82BF92BD8011696ED93FC9322243324EA
:145FEA00F801208631862286338680E090E0A0E0B0E0F90112
:145FFE0084879587A687B78780E090E0A0E0B0E0808B918BF6
:14601200A28BB38B80E090E0A0E0B0E0848B958BA68BB78B8D
:1460260080E090E0A0E0B0E0808F918FA28FB38F809104309F
:14603A0090910530892F9927907099279070E0910430F0919E
:14604E000530F070FF27FE2FEE27E070E82BF92BD8015C96EF
:14606200ED93FC938091063090910730892F99279070992744
:146076009070E0910630F0910730F070FF27FE2FEE27E0709F
:14608A00E82BF92BD8015E96ED93FC9380910830909109304C
:14609E00892F9927907099279070E0910830F0910930F070F3
:1460B200FF27FE2FEE27E070E82BF92BD8019096ED93FC93DD
:1460C60083E692E8F801E451FF4F80839183EC5EF04083E56E
:1460DA0093E6E251FF4F8083918308950E94F8DF442764E0DC
:1460EE0070E08AE99AE2FB01E80FF91F408115C04F3F19F423
:146102000FEF1FEF14C08BE99AE2FB01E80FF91F80819927ED
:146116000296680F791F8AE99AE2FB01E80FF91F40814017BC
:14612A0049F7062F172F0E9408E008952897E091B229FF274E
:14613E002080318042805380FE012082318242825382E09109
:146152008729FF272080318042805380FE0124823582468259
:1461660057826080718082809380621473048404950419F44B
:14617A0001E010E002C000271127289608950E94FCDF24978C
:14618E0003E3AADF5801C50184519F4F02961C018EEA99E204
:1461A200F101E80FF91FE081FF27408051806280738040E0DB
:1461B60050E06FEF70E0442255226622772288E090E08A9304
:1461CA00820193010E94B3EA280139018EEA99E2F101E80F2C
:1461DE00F91FE081FF27408151816281738188E190E08A93AE
:1461F2008A019B010E94B3EAA801B9014429552966297729B6
:146206008EEA99E2F101E80FF91FE081FF2740805180628096
:14621A00738080E09FEFA0E0B0E0482259226A227B2288E009
:14622E0090E08A93820193010E94A7EA402B512B622B732B73
:146242008EEA99E2F101E80FF91FE081FF27208031804280BA
:14625600538088E190E08A93810192010E94A7EA402B512B3C
:14626A00622B732BFE01408351836283738320803180428071
:14627E00538041E050E060E070E05A924A923A922A928A017D
:146292009B010E943AEB1801290156944794379427944CE3D8
:1462A60050E060E070E07A936A935A934A93810192010E9499
:1462BA006FEBFE0100831183228333834FEF5FEF60E070E0E9
:1462CE002080318042805380421553056405750538F48FEF9A
:1462E2009FEF90939C2980939B2907C0FE0120803180309282
:1462F6009C2920929B2924960E940BE008950E94E1DFE19999
:14630A00FECF4FB7F89410933F0000933E002DBBE29AE19A8E
:14631E004FBF0E94E4DF08950E94FCDF5901B8014FB7F89439
:146332002A2D8B01E6DF9501232F3327CB010196BC018C01C0
:14634600DEDF4FBF0E940BE008950E94F8DFE199FECF4FB788
:14635A00F89410933F0000933E00E09A6DB34FBF062F0E9471
:14636E0008E008950E94FCDF58016FB7F8948501E8DF402F52
:146382005527C50101965C018C01E1DF202E3324322C22243B
:14639600422953296FBF042F152F0E940BE008950E9400E0BB
:1463AA005901A80161E0CC240BC0F5016081262F8A01A3DFA7
:1463BE004F5F5F4FC50101965C01C394662319F08C2D80355E
:1463D20080F34F5F5F4F22278A0193DF0E940EE008950E94D3
:1463E600FCDF5801EF97619741E066270DC08501ACDF402FF6
:1463FA00CE01E62FFF27E80FF91F4083C50101965C01639501
:14640E00442311F0603578F36395CE01E62FFF27E80FF91F01
:146422004083AE01042F152FEF9661960E940BE008950027B0
:146436000093262F09C087E29FE2E02FFF27E80FF91F22242D
:14644A002082039588E08017A0F708950E94F8DF402F6091F8
:14645E00262F6F5F67706093262F87E29FE2E62FFF27E80FCC
:14647200F91F40838091F0438130A1F420907E27222081F4A5
:1464860020906D73222031F4242F0091E7430E94422306C030
:14649A00242F33270BE21FE10E94CFE50E9408E008950E9435
:1464AE00F8DF6091262F0AE11FE10E94CFE507E11FE10E94F2
:1464C200CFE5442715C087E29FE2E62FFF27E80FF91F2081FD
:1464D60033270BE21FE10E94CFE504E11FE10E94CFE5862F25
:1464EA0081508770682F4395483048F322242092312F2092AA
:1464FE00302F0E9408E0089587E29FE2E091262FFF27E80F37
:14651200F91F008108953A932A930E9404E0480122976627A0
:14652600772783E0C82EC4010E964C012090163030901730B7
:14653A004E845F844220532060900A3070900B306220732049
:14654E0064147504E1F420901830309019304888598842205F
:14656200532060900C3070900D30622073206414750459F4F6
:14657600288939890E851F858F939F9342D29F908F90402F42
:14658A0024C020902E1F30902F1F222091F4332081F42090CF
:14659E00301F3090311F222051F4332041F42090321F3090BA
:1465B200331F222011F4332011F041E00AC0288939890E85F7
:1465C6001F858F929F921DD29F908F90402F84E090E35C01EB
:1465DA0083E899E37C0183E0C82E1701C10102967C012501DB
:1465EE00C20102965C01F20140805180F101408251828C2D1D
:146602008150C82E882369F74E3F09F4E8C04F3F09F47BC0BA
:146616008AE0849F500182E39FE2A80EB91E8DE799E37C01B2
:14662A0083E0C82E20901630309017304E845F84422053207C
:14663E0060900A3070900B30622073206414750429F520900F
:14665200183030901930488859884220532060900C30709031
:146666000D306220732064147504A1F41701C10102967C0159
:14667A002501C20102965C01F20140805180F1014082518223
:14668E008C2D8150C82E882369F767C020902E1F30902F1F3B
:1466A200222099F4332089F42090301F3090311F222059F4A7
:1466B600332049F42090321F3090331F222019F4332009F48E
:1466CA004EC01701C10102967C0140902E1F50902F1FF10182
:1466DE00408251821C0102967C014090301F5090311FF101A0
:1466F200408251821C0102967C014090321F5090331FF10188
:14670600408251822EC08DE799E37C0183E0C82E1701C1015C
:14671A0002967C018FEF9FEFF101808391838C2D8150C82EC1
:14672E00882391F784E090E35C0183E899E37C0183E0C82E33
:146742001701C10102967C012501C20102965C01F2014080C3
:146756005180F101408251828C2D8150C82E882369F70C84BC
:14676A001D8410928A390092893980EC809344F12224209215
:14677E0045F1C4019070809346F1C401892F99279070809372
:1467920047F1209039F120FEFCCF8DE799E35C0180E09AEFC2
:1467A6006C016627772714C0FB013196EA0DFB1D2080FB0105
:1467BA00EC0DFD1D2082FB01EA0DFB1D2080FB013196EC0DAF
:1467CE00FD1D20826E5F7F4F6815790548F301E001C0002761
:1467E20022960E9411E0229608950E9404E024978DE799E3D2
:1467F6008A839B838883998384E094EF7C01A09000F4BB24D6
:14680A00A09001F4BB24BA2CAA24409102F45527209003F4D8
:14681E003324322C222442295329AA24BB241FC01701C1011E
:1468320001967C01F101608128803980C1010196888399838A
:146846002701C20101967C01F2014080F10140822880398077
:14685A00C101019688839983F1016083C50102965C01A41660
:14686E00B50608F4DDCF8091341F8F5FC82E83E18C1508F46A
:14688200CC248DE799E38A839B83EA81FB8184859585EA9370
:146896008630E8E09E07E99109F075C084899589EA938230C9
:1468AA00E0E09E07E99199F020900A3030900B3046A057A0B0
:1468BE004214530451F020900C3030900D3040A451A44214C0
:1468D200530409F057C0C092341F8AE08C9DB00182E39FE27C
:1468E600680F791FEA81FB8126803780FB0120823182EA818F
:1468FA00FB8120843184FB0122823382EA81FB81228433841C
:14690E00FB0124823582EA81FB81248C358CFB012682378267
:14692200EA81FB81268C378CFB012086318620901A30222070
:1469360039F120900E3030900F304680578042145304F1F407
:14694A0020901030309011304084518442145304A9F42080C5
:14695E00318030922F1F20922E1F228033803092311F20924C
:14697200301F248035803092331F2092321F222420921A3010
:146986000E94AB133AC0EA81FB8184859585EA938030E8E0A4
:14699A009E07E99109F02FC0C092341F8AE08C9DB00182E394
:1469AE009FE2680F791F26803780FB0120823182EA81FB81B0
:1469C20020843184FB0122823382EA81FB8122843384FB01D3
:1469D60024823582EA81FB81228C338CFB0126823782EA8134
:1469EA00FB81248C358CFB01208631868A010E5010400E9478
:1469FE00F95324960E9411E008950E94FCDFB9015801442754
:146A1200C5018F3FEFEF9E0731F46F3FEFEF7E0711F40FEF20
:146A260022C08AE0849F88E39FE2F001E80FF91F20803180B0
:146A3A00A214B30461F48AE39FE2F001E80FF91F2080318047
:146A4E006215730511F4042F0AC0842F8F5F482F853118F36A
:146A62009B0185010E9451140EEF0E940BE008950E94FCDF53
:146A76008AEF9FE25C0163E879E343E01501C10102965C011E
:146A8A002B016E5F7F4FF20140805180F10140825182842F73
:146A9E008150482F882371F71501C10102965C01F101008347
:146AB20011831C0102965C01F101208331830E940BE00895B7
:146AC6000E94E1DF45E020900E3030900F30222011F43320AE
:146ADA0001F12090103030901130222011F43320C1F081E019
:146AEE0080931A30209110303091113000910E3010910F3095
:146B02000E945114B4D020901A30222009F405C0842F815072
:146B1600482F882359F70E94E4DF08950E94E1DF44E050E33E
:146B2A0004E110E00E94984B889A909A04E110E00E94984B57
:146B3E00909804E110E00E94984B84E180930AE381E08093E8
:146B52000BE320900CE326FCFCCF0AE010E00E94984B86E3ED
:146B660080930AE381E080930BE320900CE327FEFCCF82E1C7
:146B7A0080930AE381E080930BE383ED80930CE3222420923B
:146B8E000DE388E180930AE381E080930BE320920CE380E433
:146BA20080930DE384E080930AE381E080930BE3222420921E
:146BB6000CE38DE280930DE388E580930AE381E080930BE39B
:146BCA00FA0180819181892F9927907080930CE3808191811C
:146BDE00907080930DE38AE580930AE381E080930BE38281CC
:146BF2009381892F9927907080930CE38281938190708093D7
:146C06000DE38CE580930AE381E080930BE384819581892FE4
:146C1A009927907080930CE384819581907080930DE382E222
:146C2E0080930AE3222420920BE320920CE320920DE38CE2BB
:146C420080930AE320920BE320920CE380E180930DE386E132
:146C560080930AE381E080930BE380910DE3846880930DE3D8
:146C6A000E94E4DF089588E28093E84380E18093312F809385
:146C7E00302F20901A30222031F422242092302F2092312FD9
:146C920010C080911A30813091F72090E843222071F780E2A3
:146CA6008093312F8093302F02E00E942B3208950E94FCDFFA
:146CBA00A22EA801A09762E770E30E94077A002319F4002700
:146CCE00112773C18DE090E0888399839A018E010D5E1F4F3F
:146CE2000E9478E426E83FE18E010D5E1F4F0E94D6E2A80107
:146CF60088E090E0888399839A018E010E5F1F4F0E9478E488
:146D0A0022E83FE1002711270E94D6E2A80183E090E088830B
:146D1E0099839A018E01055F1F4F0E9478E422242A862E86A1
:146D32008A2D823709F090C09E01255F3F4F8E010E5F1F4F79
:146D46003CD1A8010F3FEFEF1E0709F480C044277BC0FB0153
:146D5A00808D823009F073C088E090E0888399839E012E5F0F
:146D6E003F4F8B010E9478E483E090E0888399839E01255FDC
:146D82003F4F8B01085F1F4F0E9478E4E0913E81F0913F819F
:146D9600248C358C468C578CFB01208A318A428A538A222473
:146DAA00208E80E090E0A0E0B0E084879587A687B787E09144
:146DBE003E81F0913F81228C338C44245524FB0121A232A2E0
:146DD20043A254A2E0913E81F0913F81228C338C4424552413
:146DE600FB01218E328E438E548E222423A680E090E0A0E01C
:146DFA00B0E0848B958BA68BB78B29E030E000918081109107
:146E0E0081810E940EEBFB0101A712A7E0913E81F0913F8105
:146E2200228C338C44245524810192010E948A98FB01058FA5
:146E3600168F278F30A38B010E940E9A062F172FB8C0645D90
:146E4A007D4F4395443008F482CF00271127AFC08A2D87378C
:146E5E0009F0A9C044270AC0FB01808D813019F40027112763
:146E7200A2C0645D7D4F43954430A0F39E01255F3F4F8E01FE
:146E86000E5F1F4F9AD00F3FEFEF1E0719F0002711278FC0AB
:146E9A0062E770E3442783C0FB01808D823009F07BC000E0CB
:146EAE0010E020E030E00E94D2A1FE010787108B218B328B2A
:146EC2008FEF9FEFAFEFBFEF278430884188528828163906E1
:146ED6004A065B0619F4002711276BC0FE0127843088418835
:146EEA005288FB0121A232A243A254A2FE0127843088418821
:146EFE005288FB01218E328E438E548EFE01078510892189BA
:146F120032890E948A98FB0105A316A327A330A725A036A053
:146F260047A050A4258E368E478E50A281E0808F88E090E0F6
:146F3A00888399839E012E5F3F4F8B010E9478E483E090E005
:146F4E00888399839E01255F3F4F8B01085F1F4F0E9478E4F8
:146F620080E090E0A0E0B0E0FB01808B918BA28BB38B222467
:146F7600238680E090E0A0E0B0E084879587A687B78780E08C
:146F8A0090E0A0E0B0E0848B958BA68BB78B222423A6062F8D
:146F9E00172F0BC0645D7D4F4395443008F47ACF0027112751
:146FB20002C000271127A0960E940BE008950E94F8DFB90117
:146FC600A8019B018A010E94909A10933F8100933E81003036
:146FDA00010719F40FEF1FEF02C0002711270E9408E008953A
:146FEE000E94F8DF622FA8012497FA01808D813009F055C05A
:14700200CA010C961C01FC014080518062807380FE014082CC
:1470160051826282738281E090E0A0E0B0E0480E591E6A1E84
:14702A007B1EF1014082518262827382CA018C96FE01AF932B
:14703E00BF93A081B181FD01BF91AF91E80FF91F6083CA014E
:1470520040961C0181E090E0A0E0B0E0F101408051806280F1
:147066007380480E591E6A1E7B1E408251826282738280E067
:14707A0092E0A0E0B0E0FA0124843584468457842816390602
:14708E004A065B0661F48A010E9479A580E090E0A0E0B0E0BD
:1470A200FA0184879587A687B78701E024960E9408E008958B
:1470B6000E9400E068012497F601208C222009F068C0C60153
:1470CA000C96FC014080518062807380FE0140825182628235
:1470DE00738241E050E060E070E0440E551E661E771EFC01ED
:1470F20040825182628273824FEF51E060E070E0FE0120807E
:147106003180428053802422352246225722F101C6018C96D6
:14711A00E80FF91FA080C601449641E050E060E070E0FC01B3
:14712E004080518062807380440E551E661E771E4082518274
:1471420062827382F601208831884288538864847584868478
:147156009784261437044804590410F4AA2419C04FEF51E0D2
:14716A0060E070E0F60124843584468457842422352246227F
:14717E00572240E050E060E070E0241635064606570619F479
:1471920086010E940E9A0A2D24960E940EE008950E9400E078
:1471A6005901680168857985442755270AC01501C101019607
:1471BA005C01F1012081860115DF4F5F5F4F461757079CF3B0
:1471CE00042F152F0E940EE008950E9400E0590168016885D7
:1471E2007985442755270CC01A014F5F5F4F86012F923F9258
:1471F6005FDFFF91EF91EA0DFB1D00834617570724F486014B
:14720A004AD0002369F3042F152F0E940EE008950E9400E0B1
:14721E005901680168857985442755272DC01A014F5F5F4F63
:1472320086012F923F923EDFFF91EF91EA0DFB1D0083FA0175
:147246003197EA0DFB1D20803324C1018D30E0E09E0721F071
:14725A008A30E0E09E0791F4FA013297EA0DFB1D20803324B2
:14726E00C1018D30E0E09E0721F08A30E0E09E0719F4042FB8
:14728200152F0AC0461757072CF4860108D0002309F4CBCFF6
:14729600042F152F0E940EE00895F801208C222079F4208844
:1472AA003188428853886484758486849784621473048404F7
:1472BE00950410F001E001C0002708950E9404E06901580174
:1472D2006C9742E750E38DE090E08883998396018E01015FBF
:1472E6001F4F0E9478E426E83FE18E01015F1F4F0E94D6E243
:1472FA00B8019B018E010E5F1F4F0E947CEA22E83FE1002768
:14730E0011270E94D6E2B8019B018E01055F1F4F0E947CEA1B
:1473220022242A862E869E01255F3F4F8E010E5F1F4F45DE6F
:14733600780122E78501BCDCA8010030010709F496C0EE2061
:14734A0019F4FF2009F491C08DE090E08883998395018E018C
:14735E00015F1F4F0E9478E426E83FE18E01015F1F4F0E9422
:14737200D6E2B80188E090E0888399839B018E010E5F1F4F91
:147386000E9478E422E83FE1002711270E94D6E2B80183E0F6
:14739A0090E0888399839B018E01055F1F4F0E9478E4222407
:1473AE002A862E869E01255F3F4F8E010E5F1F4F0E94619BAE
:1473C200AA240FC02A2C33242C0C3D1CF101008111272F9270
:1473D6003F920E945A7EFF91EF910083A3948A2D8C3070F3B8
:1473EA008DE090E08883998396018E01015F1F4F0E9478E499
:1473FE0026E83FE18E01015F1F4F0E94D6E2B8019B018E01B2
:147412000E5F1F4F0E947CEA22E83FE1002711270E94D6E2A0
:14742600B8019B018E01055F1F4F0E947CEA22242A862E86EA
:14743A0088E090E0888399839E012E5F3F4F8A010E9478E4FC
:14744E0083E090E0888399839E01255F3F4F8A01085F1F4F1F
:147462000E9478E48A010E94ED9C8A0107D001E001C0002737
:147476006C960E9411E008950E94E1DFA8012497FA01208C63
:14748A002220B9F482E0808F22242082208680E090E0A0E0B0
:14749E00B0E084879587A687B78780E090E0A0E0B0E0808BCD
:1474B200918BA28BB38B01E073C0FA01808D813009F06DC04C
:1474C60080E090E0A0E0B0E02484358446845784281639064F
:1474DA004A065B0609F43BC028C0CA010C961C01FC014080C6
:1474EE00518062807380FE01408251826282738281E090E0A6
:14750200A0E0B0E0480E591E6A1E7B1EF1014082518262820C
:147516007382CA018C96FE01AF93BF93A081B181FD01BF914B
:14752A00AF91E80FF91F2224208280E092E0A0E0B0E0FA0139
:14753E002484358446845784281639064A065B0609F0C9CF74
:147552008A010E9479A5FA01018D128D238D348D0E94F5A307
:147566000E947BA18A010E94ED9C82E0FA01808F2224208249
:14757A00208680E090E0A0E0B0E084879587A687B78780E085
:14758E0090E0A0E0B0E0808B918BA28BB38B01E001C000270E
:1475A20024960E94E4DF08950E94F8DF62E770E30E94FD79EC
:1475B600002309F42DC00E94BF98402F0E94E79D442719C0E2
:1475CA002224FB012082208680E090E0A0E0B0E0848795871C
:1475DE00A687B78780E090E0A0E0B0E0808B918BA28BB38BBC
:1475F20082E0808F645D7D4F4395443028F3222420921F30D9
:14760600332430922130209220302092223008C080E28093C3
:14761A00312F8093302F05E00E942B3201E00E9408E008959E
:14762E000E94FCDFA8016E9722E78A013DDB580100300107E0
:1476420011F4002779C0F50161A172A1850116DF8DE090E06C
:14765600888399839A018E010F5E1F4F0E9478E426E83FE1C8
:14766A008E010F5E1F4F0E94D6E2A80188E090E088839983A0
:14767E009A018E010C5F1F4F0E9478E422E83FE1002711276E
:147692000E94D6E2A80183E090E0888399839A018E01035F5B
:1476A6001F4F0E9478E422242C86288A9E01235F3F4F8E017C
:1476BA000C5F1F4F0E94619B002311F4002738C020901C3002
:1476CE00222019F04FEF5FE01EC04FEF5FEF1BC05B016030AF
:1476E200670711F4002728C01B0144245524810192010E945E
:1476F600909EB801150144245524288239824A825B8200E0B4
:14770A0010E020E030E00E943AA26417750711F71501442470
:14771E005524288239824A825B8200E010E020E030E00E944E
:147732003AA20E947BA101E06E960E940BE00895F801048914
:1477460015892689378908953A932A930E9400E058012F975A
:14775A008B8D9C8D8130E0E09E0751F00B8C1C8C002011F41F
:14776E00112021F0F501808D823019F40FEF1FEF3EC088E091
:1477820090E08883998395018E010E5F1F4F0E9478E48EE2EE
:147796008A8783E090E0888399839501285F3F4F8E01055F36
:1477AA001F4F0E9478E422242E86F501208C222019F482E70B
:1477BE00C82E02C087E7C82E85015ADE2C2D8E010E5F1F4F1A
:1477D20071DA02C085016EDCFE012788308C418C528CF501BB
:1477E600648875888688978862147304840495047CF30027D5
:1477FA0011272F960E940EE02296089520901F30222061F403
:14780E0022243324309221302092203081E080931F300FE101
:1478220010E302C00027112708950E94E1DFA801659740302A
:14783600450721F0FA012080222019F40027112778C0CA0195
:14784A000196FC0140805180C20101968083918382010E946F
:14785E007E9C10933F8100933E81E0913E81F0913F81208036
:147872003324C101EA93853EE0E09E07E99119F3EA9385308C
:14788600E0E09E07E991E9F223843324C101EA938230E0E085
:14789A009E07E991A1F2EA938F30E0E09E07E99109F4CDCF74
:1478AE00E030EF0719F4002711273FC0E0913E81F0913F81E4
:1478C200248C358C468C578CFE01218A328A438A548A88E013
:1478D60090E08883998320913E8130913F818E010C5F1F4FAE
:1478EA000E9478E422242C8683E090E08883998320913E812A
:1478FE0030913F81285F3F4F8E01035F1F4F0E9478E422243D
:14791200288ACE010D968A839B83CE0104968883998329E772
:147926003FE18A010D5F1F4F0E942BE38A010D5F1F4F6596B8
:14793A000E94E4DF08950E94F8DFB801ED970E94077A00233B
:14794E0031F4222420921B3000271127CFC06030670721F0C0
:14796200FB012080222031F4222420921B3000271127C2C0EA
:14797600CB010196FC0140805180C201019680839183820118
:14798A000E947E9C10933F8100933E81E0913E81F0913F8107
:14799E0020803324C101EA93853EE0E09E07E99119F3EA9374
:1479B2008530E0E09E07E991E9F223843324C1018230E0E020
:1479C6009E07B1F28F30E0E09E0709F4D1CF20901B30222067
:1479DA0031F0222420921B300027112789C020903E8130905E
:1479EE003F81222001F53320F1F481E080931B300E9412A63C
:147A0200FE010787108B218B328BCE0147968883998387D0B5
:147A1600CE0147968883998328E63FE18B010D5F1F4F0E9453
:147A2A002BE38B010D5F1F4F63C0222420921B30E0913E813E
:147A3E00F0913F814385248C358C468C578CFE012786308A9F
:147A5200418A528ACE01C5968883998307851089218932899E
:147A66005ED088E090E08883998320913E8130913F818E015F
:147A7A000A5F1F4F0E9478E4442712C0CE010696E42FFF2742
:147A8E00E80FF91F8081803241F4CE010696E42FFF27E80F52
:147AA200F91F22242082439587E0841758F722242E862091FC
:147AB6003E8130913F81285F3F4F8E010D5E1F4F0E947CEAF7
:147ACA0022242E8ACE0143968C839D83CE0106968A839B833D
:147ADE00CE01C5968883998325E33FE18B010D5F1F4F0E9413
:147AF2002BE38B010D5F1F4FED960E9408E0089522243324C5
:147B0600F801218232820895F8012080222011F4002704C0B3
:147B1A002224F801208201E008950E947FDF0E9404E02497B7
:147B2E00AA24CC24C39440E051EE65EF75E0FE014083518390
:147B42006283738359C0FE0120803180428053806684778471
:147B5600808891885A924A923A922A92830194010E946FEB95
:147B6A00E02EFE0120803180428053806E2C77248824992476
:147B7E005A924A923A922A92830194010E943AEBFE0126841A
:147B9200378440885188201A310A420A530A26863786408A32
:147BA600518A8E2D805DE82E803311F4CC2061F42A2C33249C
:147BBA008A2D8F5FA82EF1010A881B88E00DF11DE082CC24C8
:147BCE004AE050E060E070E0FE0120803180428053807A93C7
:147BE2006A935A934A93810192010E946FEBFE0100831183A1
:147BF6002283338340E050E060E070E0FE012080318042802E
:147C0A005380241635064606570609F098CFEA2DFF270A8846
:147C1E001B88E00DF11D2224208224960E9411E02496089528
:147C32000E9404E0EF97EF97EF97EF97EF97EF97EF97EF9788
:147C4600E4970E94C84A40E050E060E070E068837983242FE1
:147C5A00352F05E110E00E94B194002309F052C040E050E077
:147C6E0060E070E068837983242F352F05E110E00E943F938A
:147C820022242092303984E080933139209232393324309276
:147C960036392092353940E050E060E070E050933A39409342
:147CAA00393970933C3960933B3940E050E060E070E05093B2
:147CBE003E3940933D397093403960933F3930923839209226
:147CD200373930924239209241393092443920924339309296
:147CE60056392092553930925839209257392090B4473090BB
:147CFA00B547309234392092333922242092453920924D397F
:147D0E0080E399E3FE01EE5DFD4F8083918305E110E00E945D
:147D22002093FE01E05EFD4F008311830C947B4A2090353977
:147D360030903639DE01A05EBD4FED91FC9145805680421425
:147D4A00530419F540903B3950903C392090393930903A39D2
:147D5E006180728088249924621473048404950491F4409072
:147D72003F395090403920903D3930903E396380748088244C
:147D86009924621473048404950409F4A4C020903039222062
:147D9A0009F07FC0DE01A05EBD4FED91FC918285823009F0F7
:147DAE0076C081E0DE01AE5DBD4FED91FC918083DE01A05E49
:147DC200BD4FED91FC912180328044245524DE01AE5DBD4F6C
:147DD600ED91FC912186328643865486DE01A05EBD4FED9125
:147DEA00FC912380348044245524DE01AE5DBD4FED91FC91BF
:147DFE00258636864786508ADE01A05EBD4FED91FC912580CA
:147E12003680DE01AE5DBD4FED91FC912582368222243324A9
:147E2600DE01AE5DBD4FED91FC9127823086DE01AE5DBD4FF2
:147E3A00ED91FC91218A328ADE01AE5DBD4FED91FC91238A14
:147E4E00348A2090B4473090B547DE01AE5DBD4FED91FC91FA
:147E620023823482DE01AE5DBD4FED91FC91DE01A05EBD4FC7
:147E76000D901C9003A614A682EC98E08883998321E430E02A
:147E8A00FE01E05EFD4F008111810E940E970C946F4ADE01C9
:147E9E00A05EBD4FED91FC918285823011F00C946F4A83E045
:147EB20099E0888399832AE130E0FE01E05EFD4F0081118165
:147EC6000E940E97FE01E05EFD4F008111810E94AF970C943D
:147EDA006F4ADE01A05EBD4FED91FC918285833049F4FE01F1
:147EEE00E05EFD4F008111810E94AF970C946F4AFE01E05E65
:147F0200FD4F008111810E945C960030010709F4C6C78091A5
:147F16003039843009F4C1C7DE01A05EBD4FED91FC918285BA
:147F2A00823009F0B8C781E08A83CE0104968883998320E01B
:147F3E0031E0FE01E05EFD4F008111810E94F495FE01E85D13
:147F5200FD4F00831183CE010496DE01A85DBD4FED91FC9154
:147F66003197E80FF91F20803324C1018D30E0E09E0731F034
:147F7A008A30E0E09E0711F00C946F4A2090B4473090B54713
:147F8E00DE01AE5DBD4FED91FC9123823482FE01E05EFD4FFA
:147FA200008111810E947596CE010496DE01A85DBD4FED9134
:147FB600FC91E80FF91F2224208220ED3FE18E010C5F1F4F9E
:147FCA000E94D6E2FE01EA5DFD4F0083118300241124FE0148
:147FDE00EC5DFD4F0082118221C0FE01EC5DFD4F208031801F
:147FF200FE01EA5DFD4F00801180200C311CF10100811127B4
:148006002F923F920E945A7EFF91EF910083FE01EC5DFD4F33
:14801A00808191810196FE01EC5DFD4F80839183FE01EA5DB7
:14802E00FD4F008111810E9426E5FE01EC5DFD4F008011808D
:148042000016110680F2DE01AE5DBD4FED91FC91E080FF2407
:14805600C7018130E0E09E0761F08230E0E09E0709F46CC0A7
:14806A008330E0E09E0709F4E1C00C946F4A2BEC3FE1FE01BD
:14807E00EA5DFD4F008111810E9485E30030010711F00C9465
:148092006F4A20ED3FE1002711270E94D6E2FE01EA5DFD4FA9
:1480A600008311838DE199E0888399832BE130E0FE01E05E48
:1480BA00FD4F008111810E940E97FE01EA5DFD4F0081118167
:1480CE000E9426E51801FE01EA5DFD4F008011800882198210
:1480E2009101FE01E05EFD4F008111810E949A9687EC9FE197
:1480F6008883998323E030E0FE01E05EFD4F008111810E94FE
:14810A009A9688E090E088839983FE01EA5DFD4F208131814D
:14811E00FE01EE5DFD4F008111810B5E1F4F0E9478E482E06D
:14813200DE01AE5DBD4FED91FC9180830C946F4A22EC3FE1AE
:14814600FE01EA5DFD4F008111810E9485E30030010711F03D
:14815A000C946F4A20ED3FE1002711270E94D6E2FE01EA5D8C
:14816E00FD4F0083118388E090E088839983FE01EA5DFD4F09
:1481820020813181FE01EE5DFD4F00811181035E1F4F0E947C
:1481960078E4FE01EE5DFD4F20813181235E3F4F07EE16E492
:1481AA000E9485E30030010771F4FE01EE5DFD4F2081318131
:1481BE002B5E3F4F0BEF16E40E9485E300300107E9F08EE415
:1481D20099E08883998327E130E0FE01E05EFD4F0081118145
:1481E6000E940E97FE01E05EFD4F008111810E94AF97FE01BB
:1481FA00EE5DFD4F008111810E94944A0C946F4A88E399E00A
:14820E008883998326E130E0FE01E05EFD4F008111810E94E0
:148222000E9783E0DE01AE5DBD4FED91FC9180830C946F4AE3
:148236002DEB3FE1FE01EA5DFD4F008111810E9485E300301D
:14824A000107E9F485E699E08883998323E230E0FE01E05EDE
:14825E00FD4F008111810E940E97FE01E05EFD4F00811181CA
:148272000E94AF97FE01EE5DFD4F008111810E94944A0C9447
:148286006F4A28EB3FE1FE01EA5DFD4F008111810E9485E349
:14829A000030010709F074C020ED3FE1002711270E94D6E285
:1482AE00FE01EA5DFD4F00831183DE01AA5DBD4FED91FC9116
:1482C200008111270E945A7E202EDE01AA5DBD4FED91FC912A
:1482D6002082DE01AA5DBD4FED91FC9180818134B1F4222454
:1482EA00DE01AE5DBD4FED91FC9122828DE999E088839983C5
:1482FE0025E130E0FE01E05EFD4F008111810E940E970C94D3
:148312006F4ADE01AA5DBD4FED91FC9180818934B1F481E0DD
:14832600DE01AE5DBD4FED91FC91828388E899E0888399832D
:14833A0025E130E0FE01E05EFD4F008111810E940E970C9496
:14834E006F4A82EB99E0888399832EE130E0FE01E05EFD4FAD
:14836200008111810E940E97FE01E05EFD4F008111810E946F
:14837600AF97FE01EE5DFD4F008111810E94944A0C946F4A2B
:14838A0023EB3FE1FE01EA5DFD4F008111810E9485E30030D2
:14839E00010709F001C121EB3FE1002711270E94D6E2FE0124
:1483B200EA5DFD4F00831183FE01EA5DFD4F0080118000204A
:1483C60019F4112009F4C6C00E947AE51801322C2224DE0145
:1483DA00AE5DBD4FED91FC91218A328A21EB3FE1002711277B
:1483EE000E94D6E2FE01EA5DFD4F00831183FE01EA5DFD4FE6
:1484020000801180002019F4112009F4A5C00E947AE5FE0195
:14841600EE5DFD4F808191814196FC0160807180602A712ADE
:14842A006082718221EB3FE1002711270E94D6E2FE01EA5D3E
:14843E00FD4F00831183FE01EA5DFD4F00801180002019F4F7
:14845200112009F481C00E947AE51801322C2224DE01AE5DFF
:14846600BD4FED91FC91238A348A21EB3FE1002711270E9453
:14847A00D6E2FE01EA5DFD4F00831183FE01EA5DFD4F00807B
:14848E001180002019F4112009F460C00E947AE5FE01EE5D83
:1484A200FD4F808191814396FC0160807180602A712A6082B9
:1484B600718221EB3FE1002711270E94D6E2FE01EA5DFD4F48
:1484CA0000831183FE01EA5DFD4F00801180002019F4112086
:1484DE0009F43CC00E947AE51801322C2224DE01AE5DBD4FDD
:1484F200ED91FC912782308620ED3FE1002711270E94D6E226
:14850600FE01EA5DFD4F00831183FE01EA5DFD4F0080118015
:14851A00002011F41120E1F00E947AE5FE01EE5DFD4F80818E
:14852E0091810796FC0160807180602A712A6082718280ED55
:1485420099E0888399832FE130E0FE01E05EFD4F00811181C9
:148556000E940E97FE01EA5DFD4F00801180002009F0BAC78D
:14856A00112009F0B7C782EB99E0888399832EE130E0FE012A
:14857E00E05EFD4F008111810E940E97FE01E05EFD4F0081FB
:1485920011810E94AF97FE01EE5DFD4F00811181C2D79CC7B6
:1485A6002DEA3FE1FE01EA5DFD4F008111810E9485E30030AB
:1485BA00010771F48FEE99E08883998320E230E0FE01E05ED4
:1485CE00FD4F008111810E940E9782C728EA3FE1FE01EA5D32
:1485E200FD4F008111810E9485E30030010769F023EA3FE15E
:1485F600FE01EA5DFD4F008111810E9485E30030010709F091
:14860A0021C1DE01AE5DBD4FED91FC912280222071F48FE0C1
:14861E009AE0888399832DE130E0FE01E05EFD4F00811181ED
:148632000E940E970DC08CE29AE0888399832EE130E0FE01F3
:14864600E05EFD4F008111810E940E9784E190E08A839B833C
:14865A00DE01AE5DBD4FED91FC912388348828823982DE0160
:14866E00AE5DBD4FED91FC9121893289078110850E949D9382
:148682001801DE01AE5DBD4FED91FC9121A632A6DE01AE5D41
:14869600BD4FED91FC9121A432A4222081F4332071F48AE441
:1486AA009AE08883998326E230E0FE01E05EFD4F0081118167
:1486BE000E940E970DC70E94033C1801DE01AE5DBD4FED911F
:1486D200FC9127A230A6DE01AE5DBD4FED91FC9127A030A4CC
:1486E600222019F4332009F4A1C084E0808323EA3FE1FE01ED
:1486FA00EA5DFD4F008111810E9485E300300107B1F4222499
:14870E00DE01AE5DBD4FED91FC912182DE01AE5DBD4FED913F
:14872200FC9107A110A50E94163CFE01EA5DFD4F00831183BC
:1487360015C081E0DE01AE5DBD4FED91FC918183DE01AE5D0A
:14874A00BD4FED91FC9107A110A50E94A03CFE01EA5DFD4F97
:14875E0000831183FE01EA5DFD4F00801180002011F41120F7
:14877200D1F0FE01EA5DFD4F008111810E9426E51801FE01C8
:14878600EA5DFD4F00801180088219829101DE01AE5DBD4F8E
:14879A00ED91FC9101A512A50E949A969BC6DE01AE5DBD4F3A
:1487AE00ED91FC9101A512A50E94AF9780E79AE0888399835F
:1487C20020E230E0FE01E05EFD4F008111810E940E9783E04B
:1487D600DE01AE5DBD4FED91FC91808384E0DE01AE5DBD4F31
:1487EA00ED91FC91818322243324DE01AE5DBD4FED91FC91CE
:1487FE0027823086DE01AE5DBD4FED91FC91218A328ADE01C1
:14881200AE5DBD4FED91FC91238A348ADE01AE5DBD4FED9151
:14882600FC9107A110A50E94873D56C680E79AE088839983CA
:14883A0020E230E0FE01E05EFD4F008111810E940E9748C627
:14884E002EE93FE1FE01EA5DFD4F008111810E9485E3003000
:14886200010709F000C120ED3FE1002711270E94D6E2FE015B
:14887600EA5DFD4F008311832CE93FE10E94D6E2680188E0E4
:14888A0090E08883998396018E010C5F1E4F0E9478E4222401
:14889E00FE01E45FFE4F20822CE93FE18E010C5F1E4F0E9457
:1488B20002E520ED3FE1002711270E94D6E2680183E090E0A9
:1488C6008883998396018E010C5F1E4F0E9432E522E78E0128
:1488DA000C5F1E4F0E945B361801DE01AE5DBD4FED91FC9165
:1488EE0025A236A2DE01AE5DBD4FED91FC9125A036A02220F9
:1489020019F4332009F4A1C02280222071F48FE09AE0888366
:1489160099832DE130E0FE01E05EFD4F008111810E940E9730
:14892A000DC08CE29AE0888399832EE130E0FE01E05EFD4FB5
:14893E00008111810E940E9784E190E08A839B83DE01AE5DE1
:14895200BD4FED91FC912388348828823982DE01AE5DBD4F38
:14896600ED91FC9121893289078110850E949D931801DE01A6
:14897A00AE5DBD4FED91FC9121A632A6DE01AE5DBD4FED91B4
:14898E00FC9121A432A42220C9F43320B9F48AE49AE08883BB
:1489A200998326E230E0FE01E05EFD4F008111810E940E97AA
:1489B600DE01AE5DBD4FED91FC9105A116A10E943F3A8AC5E5
:1489CA0084E0DE01AE5DBD4FED91FC91808382E0DE01AE5DE5
:1489DE00BD4FED91FC91818380E091E0888399839E012E5E47
:1489F2003E4FDE01AE5DBD4FED91FC9105A116A10E94EC38C0
:148A0600FE01EC5DFD4F00831183FE01EC5DFD4F008011800C
:148A1A00002019F4112009F45DC5CE018E5E9E4F88839983FC
:148A2E00FE01EC5DFD4F20813181DE01AE5DBD4FED91FC914C
:148A420001A512A50E949A9649C580E99AE0888399832BE1CD
:148A560030E0FE01E05EFD4F008111810E940E973BC527E909
:148A6A003FE1FE01EA5DFD4F008111810E9485E300300107F1
:148A7E0009F0D6C08FEF8093982020ED3FE1002711270E94DE
:148A9200D6E2FE01EA5DFD4F008311832CE93FE10E94D6E2E0
:148AA600680188E090E08883998396018E010C5F1E4F0E94B4
:148ABA0078E42224FE01E45FFE4F20822CE93FE18E010C5FA6
:148ACE001E4F0E9402E520ED3FE1002711270E94D6E268014F
:148AE20083E090E08883998396018E010C5F1E4F0E9432E5CF
:148AF6008E010C5F1E4F0E94173B27E78E010C5F1E4F0E94FA
:148B0A005B361801DE01AE5DBD4FED91FC9125A236A2DE012E
:148B1E00AE5DBD4FED91FC9125A036A0222019F4332009F4E7
:148B32006FC02280222071F48FE09AE0888399832DE130E089
:148B4600FE01E05EFD4F008111810E940E970DC08CE29AE083
:148B5A00888399832EE130E0FE01E05EFD4F008111810E9483
:148B6E000E9784E190E08A839B83DE01AE5DBD4FED91FC914D
:148B82002388348828823982DE01AE5DBD4FED91FC91218968
:148B96003289078110850E949D931801DE01AE5DBD4FED9194
:148BAA00FC9121A632A6DE01AE5DBD4FED91FC9121A432A4EF
:148BBE002220C9F43320B9F48AE49AE08883998326E230E07D
:148BD200FE01E05EFD4F008111810E940E97DE01AE5DBD4FB6
:148BE600ED91FC9105A116A10E943F3A75C484E0DE01AE5D71
:148BFA00BD4FED91FC91808383E0DE01AE5DBD4FED91FC91E9
:148C0E00818366C480E99AE0888399832BE130E0FE01E05EC1
:148C2200FD4F008111810E940E9758C422E93FE1FE01EA5D0B
:148C3600FD4F008111810E9485E30030010709F05AC020ED69
:148C4A003FE1002711270E94D6E2FE01EA5DFD4F0083118394
:148C5E002CE93FE10E94D6E2680188E090E088839983960174
:148C72008E010C5F1E4F0E9478E42224FE01E45FFE4F208212
:148C86002CE93FE18E010C5F1E4F0E9402E520ED3FE1002761
:148C9A0011270E94D6E2680183E090E08883998396018E01AB
:148CAE000C5F1E4F0E9432E58E010C5F1E4F0E94173B0023A3
:148CC20071F08BEA9AE0888399832AE130E0FE01E05EFD4F83
:148CD600008111810E940E97FFC380E99AE0888399832BE158
:148CEA0030E0FE01E05EFD4F008111810E940E97F1C32DE8BA
:148CFE003FE1FE01EA5DFD4F008111810E9485E3003001075B
:148D120009F04EC020ED3FE1002711270E94D6E2FE01EA5D1A
:148D2600FD4F008311832CE93FE10E94D6E2680188E090E006
:148D3A0088839983960102E219E30E9478E4222420922A392E
:148D4E002CE93FE102E219E30E9402E520ED3FE100271127E7
:148D62000E94D6E2680183E090E088839983960102E219E3C9
:148D76000E9432E585EC9AE08883998326E330E0FE01E05EC8
:148D8A00FD4F008111810E940E97A4C380E99AE088839983BE
:148D9E002BE130E0FE01E05EFD4F008111810E940E9796C369
:148DB20028E83FE1FE01EA5DFD4F008111810E9485E300309E
:148DC600010709F05CC020ED3FE1002711270E94D6E2FE0197
:148DDA00EA5DFD4F008311832CE93FE10E94D6E2680188E07B
:148DEE0090E08883998396018E010E5E1D4F0E9478E4222498
:148E0200FE01E65EFD4F20822CE93FE18E010E5E1D4F0E94ED
:148E160002E520ED3FE1002711270E94D6E2680183E090E03F
:148E2A008883998396018E010E5E1D4F0E9432E59E012E5E2B
:148E3E003D4F02E219E30E946539002371F08BEA9AE08883F6
:148E520099832AE130E0FE01E05EFD4F008111810E940E97F2
:148E66003BC380E99AE0888399832BE130E0FE01E05EFD4F4B
:148E7A00008111810E940E972DC382EB99E0888399832EE17E
:148E8E0030E0FE01E05EFD4F008111810E940E971FC3DE011C
:148EA200AE5DBD4FED91FC918081843009F016C321A432A478
:148EB600222019F4332009F40FC343885488F10163807480C7
:148ECA006414750409F0F8C2DE01AE5DBD4FED91FC91418826
:148EDE005288F101618072806414750409F0EAC2DE01AE5D61
:148EF200BD4FED91FC9147805084F1012580368024143504FC
:148F060009F0DCC2DE01AE5DBD4FED91FC91A180BB24AA20F5
:148F1A0011F4BB2081F0C5018130E0E09E0759F08230E0E05B
:148F2E009E0709F4ACC08330E0E09E0709F45FC194C2DE01B7
:148F4200AE5DBD4FED91FC9127A030A4222019F4332009F4BF
:148F560075C02090B4473090B54723823482DE01AE5DBD4F1A
:148F6A00ED91FC91AF93BF93A1A5B2A5FD01BF91AF91828522
:148F7E00823009F0ADC2DE01AE5DBD4FED91FC9121802220E1
:148F920051F407A110A50E94163CFE01EA5DFD4F008311838C
:148FA6000EC0DE01AE5DBD4FED91FC9107A110A50E94A03C0D
:148FBA00FE01EA5DFD4F00831183FE01EA5DFD4F0080118057
:148FCE000020F1F41120E1F4DE01AE5DBD4FED91FC9107A1DB
:148FE20010A50E94873DDE01AE5DBD4FED91FC9101A512A502
:148FF6000E94AF9722243324DE01AE5DBD4FED91FC9127A218
:14900A0030A668C2FE01EA5DFD4F008111810E9426E51801E7
:14901E00FE01EA5DFD4F00801180088219829101DE01AE5DFA
:14903200BD4FED91FC9101A512A50E949A964EC28BEF9AE0E0
:149046008883998329E130E0FE01E05EFD4F008111810E9497
:14905A000E9722243324DE01AE5DBD4FED91FC9121A632A620
:14906E0083E0DE01AE5DBD4FED91FC91808384E0DE01AE5D39
:14908200BD4FED91FC91818329C2DE01AE5DBD4FED91FC91D3
:1490960025A036A0222019F4332009F487C02090B4473090DA
:1490AA00B54723823482DE01AE5DBD4FED91FC91AF93BF93C6
:1490BE00A1A5B2A5FD01BF91AF918285823009F007C2DE0119
:1490D200AE5DBD4FED91FC9105A116A10E945039002309F0C4
:1490E60049C0DE01AE5DBD4FED91FC9101A512A50E94659672
:1490FA00FE01E65DFD4F0083118380E091E0FE01E65DFD4F5E
:14910E00008011808015910528F4FE01E65DFD4F8083918350
:14912200FE01E65DFD4F00801180088219829E012E5E3E4FBD
:14913600DE01AE5DBD4FED91FC9105A116A10E94EC38FE0102
:14914A00EC5DFD4F00831183CE018E5E9E4F88839983FE0197
:14915E00EC5DFD4F20813181DE01AE5DBD4FED91FC9101A56E
:1491720012A50E949A96B2C1DE01AE5DBD4FED91FC9105A146
:1491860016A10E943F3A22243324DE01AE5DBD4FED91FC9165
:14919A0025A236A2DE01AE5DBD4FED91FC9101A512A50E9422
:1491AE00AF9796C18BEF9AE08883998329E130E0FE01E05E9E
:1491C200FD4F008111810E940E9722243324DE01AE5DBD4F60
:1491D600ED91FC9121A632A683E0DE01AE5DBD4FED91FC9177
:1491EA00808384E0DE01AE5DBD4FED91FC91818371C1DE01F4
:1491FE00AE5DBD4FED91FC9125A036A0222019F4332009F401
:14921200FCC02090B4473090B54723823482DE01AE5DBD4FD4
:14922600ED91FC9121A432A4222019F4332009F4C9C0CE0197
:14923A0004968883998320E031E0DE01AE5DBD4FED91FC914D
:14924E0001A512A50E94DD94FE01E65DFD4F00831183FE01F8
:14926200E65DFD4F00801180002019F4112009F461C0088252
:1492760019829E012C5F3F4FDE01AE5DBD4FED91FC9105A1EA
:14928A0016A10E94D138FE01EC5DFD4F00831183FE01EC5D7B
:14929E00FD4F00801180FE01E65DFD4F008111810016110691
:1492B20009F440C080E99AE0888399832BE130E0FE01E05E48
:1492C600FD4F008111810E940E97DE01AE5DBD4FED91FC91ED
:1492DA0001A512A50E94AF9722243324DE01AE5DBD4FED912A
:1492EE00FC9121A632A683E0DE01AE5DBD4FED91FC918083D9
:1493020084E0DE01AE5DBD4FED91FC918183DE01AE5DBD4FF8
:14931600ED91FC9105A116A10E943F3ADE01AE5DBD4FED914C
:14932A00FC9101A512A50E94AF97D4C0DE01AE5DBD4FED9155
:14933E00FC9121A432A4F1018285833009F0C8C081010E94A2
:149352005C960030010709F0C1C0DE01AE5DBD4FED91FC9162
:1493660005A116A10E943F3ADE01AE5DBD4FED91FC9101A5D4
:14937A0012A50E94AF9722243324DE01AE5DBD4FED91FC91A2
:14938E0021A632A683E0DE01AE5DBD4FED91FC91808384E061
:1493A200DE01AE5DBD4FED91FC9181838BEF9AE08883998397
:1493B60029E130E0FE01E05EFD4F008111810E940E978AC05C
:1493CA00DE01AE5DBD4FED91FC9101A512A50E94AF97222403
:1493DE003324DE01AE5DBD4FED91FC9121A632A683E0DE0142
:1493F200AE5DBD4FED91FC91808384E0DE01AE5DBD4FED916A
:14940600FC91818369C080E99AE0888399832BE130E0FE0173
:14941A00E05EFD4F008111810E940E97DE01AE5DBD4FED91E6
:14942E00FC9101A512A50E94AF9722243324DE01AE5DBD4FC5
:14944200ED91FC9121A632A683E0DE01AE5DBD4FED91FC9108
:14945600808384E0DE01AE5DBD4FED91FC9181833BC0222455
:14946A003324DE01AE5DBD4FED91FC9121A632A6DE01AE5D0D
:14947E00BD4FED91FC9127823086DE01AE5DBD4FED91FC9163
:14949200218A328ADE01AE5DBD4FED91FC91238A348A83E090
:1494A600DE01AE5DBD4FED91FC91808384E0DE01AE5DBD4F54
:1494BA00ED91FC9181830EC084E0DE01AE5DBD4FED91FC915C
:1494CE00818383E0DE01AE5DBD4FED91FC918083DE01A05E42
:1494E200BD4FED91FC9123843484FE01E05EFD4F2082318222
:1494F600FE01E05EFD4F00801180002011F00C94993E1120FF
:14950A0011F00C94993EEF96EF96EF96EF96EF96EF96EF9632
:14951E00EF96E4960E9411E0089522243324F8012782308615
:14953200208284E08183222422822582368280E090E0A0E082
:14954600B0E081879287A387B48780E090E0A0E0B0E085870F
:14955A009687A787B08B222427823086218A328A238A348A00
:14956E0025A236A227A230A62090B4473090B54723823482E9
:149582002224258A258E81E08093982008950E94F8DF20903B
:149596003039222009F4C6C0E0915B39F0915C392180328025
:1495AA004424552480903B3990903C396090393970903A39DE
:1495BE006214730484049504D1F4238034804424552480907E
:1495D2003F399090403960903D3970903E3962147304840422
:1495E600950449F42580368040903539509036394214530406
:1495FA00F1F122242092303984E080933139209232393324C5
:14960E00309236392092353940E050E060E070E050933A39C1
:149622004093393970933C3960933B3940E050E060E070E030
:1496360050933E3940933D397093403960933F393092383963
:14964A00209237393092423920924139309244392092433914
:14965E003092563920925539309258392092573920924539A2
:1496720020924D393BC0809130398430B9F5E0915939F09151
:149686005A392180328040904139509042394214530491F413
:14969A002380348040904339509044394214530449F425802D
:1496AE003680409037395090383942145304C1F02224332466
:1496C20030925A392092593983E08093303984E0809331393B
:1496D600309238392092373930924239209241393092443983
:1496EA0020924339E0915B39F0915C398285833021F48F01C4
:1496FE000E94AF9713C02090B4473090B54780913339909198
:1497120034398059984E8215930531F400915B3910915C3968
:149726000E94DC970E9408E008950E94E1DF43E357E0CA0169
:14973A000197AC0180308907D1F7C80101978C0180308907A0
:14974E0091F70E94E4DF08950E94FCDF44275527B801FB0164
:149762008081803309F048C021803324C1018837E0E09E0760
:1497760029F08835E0E09E0709F03CC06E5F7F4F39C0C50155
:14978A008033E0E09E0748F089E390E08A159B0520F0C5018A
:14979E00C0975C011FC0C5018136E0E09E0758F086E690E01E
:1497B2008A159B0530F0C501815690400A965C010FC0C50145
:1497C6008134E0E09E0718F186E490E08A159B05F0F0C501AD
:1497DA00815490400A965C011A01220C331C220C331C220C96
:1497EE00331C220C331C2A0C3B1CA1011B016F5F7F4FF101C2
:14980200208033245101222009F0BDCF332009F0BACF042F3A
:14981600152F0E940BE0089500273EC08DE599E3E02FFF2788
:14982A00EE0FFF1FEE0FFF1FEE0FFF1FE80FF91F222433242D
:14983E00208231828FE599E3E02FFF27EE0FFF1FEE0FFF1F66
:14985200EE0FFF1FE80FF91F22242082318281E699E3E02F4B
:14986600FF27EE0FFF1FEE0FFF1FEE0FFF1FE80FF91F222422
:14987A002082318283E699E3E02FFF27EE0FFF1FEE0FFF1F35
:14988E00EE0FFF1FE80FF91F2224208231820395043008F439
:1498A200BFCF08950E94E1DF229780E090E0A0E0B0E0A88361
:1498B600B983282F392F00E510E00E94B194002369F480E007
:1498CA0090E0A0E0B0E0A883B983282F392F00E510E00E946D
:1498DE003F9310C000E510E00E942093A80107C08A01BAD025
:1498F2008A010AD0FA014385548540304507B1F722960E94A3
:14990600E4DF08950E94FCDFB801EF97A7978DE599E3FB0109
:14991A0040815527440F551F440F551F440F551F480F591FD8
:14992E00FA0126803780222019F4332009F48FC0208031808E
:14994200FB014580568042145304A9F4FA0122803380FB01E4
:14995600418052804214530461F4FA0124803580FB01438055
:14996A0054804214530419F48285843059F4FA010681178139
:14997E000E943F3A22243324FA012682378267C0FB01828597
:14999200833071F48B010E94AF97FA01068117810E943F3A00
:1499A60022243324FA012682378255C0FA01068117810E94E3
:1499BA005039002309F030C08B010E9465960436E0E01E07BC
:1499CE007CF48B010E946596088319839E012E5F3F4FFA0110
:1499E200068117810E94EC3858010DC084E690E08883998365
:1499F6009E012E5F3F4FFA01068117810E94EC385801AA20A0
:149A0A0011F4BB2031F1CE0102968883998395018B010E94F4
:149A1E009A961DC02BE53CE08E010E5F1F4F0E94067FCE019B
:149A320002968883998322E030E08B010E949A968B010E94C3
:149A4600AF97FA01068117810E943F3A22243324FA01268251
:149A5A003782EF96A7960E940BE008951A930A930E9404E083
:149A6E00EF97EF97EF97EF97EF97EF97EF97EF97EF97EF97A8
:149A8200E597CC2422243324FE01E057FD4F20823182FE01F1
:149A9600EB54FD4F008111810E945C960030010709F4EAC2A9
:149AAA0083E699E3DE01AB54BD4FED91FC91E081FF27EE0F4A
:149ABE00FF1FEE0FFF1FEE0FFF1FE80FF91F2080318022209E
:149AD20009F0D4C2332009F0D1C281E08A83CE01069688832E
:149AE60099832AE832E0FE01EB54FD4F008111810E94F49564
:149AFA00B8010030010711F1CE010696FB013197E80FF91F27
:149B0E0020803324C1018D30E0E09E07B1F08A30E0E09E07A8
:149B220091F0CE010696FB013297E80FF91F20803324C101B6
:149B36008D30E0E09E0729F08A30E0E09E0709F09BC281E00A
:149B4A008A83CE010696888399832AE832E0FE01EB54FD4FBA
:149B5E00008111810E94C295B80122E930E28E010A5F1F4FAB
:149B72000E94D6E2580183E090E0888399832DE830E20E9469
:149B860035E40030010709F05BC1FE01EB54FD4F00811181C8
:149B9A000E9475962AE830E2002711270E94D6E2A8010E94E2
:149BAE0026E5E02E22E930E28A010E94D6E2A8010E9426E532
:149BC2002E2C33242016310619F4CC24C39440C022E930E200
:149BD600002711270E94D6E2780188E090E08883998321E841
:149BEA0030E20E9435E40030010719F4CC24C3942BC088E0BB
:149BFE0090E08883998328E730E287010E9435E40030010720
:149C1200F9F088E090E0888399832FE630E287010E9435E4EC
:149C26000030010799F081E08C83FE01EB54FD4F008011805E
:149C3A000A821B8287E19DE08883998325EA3CE006E21BE0D3
:149C4E0026D216C282E090E0888399832CE630E28A010E94E8
:149C620035E40030010771F48AE697E28883998327E630E209
:149C76008E010E561D4F0E942BE3AE014E565D4F8BE090E0F1
:149C8A008883998328E530E28A010E9435E400300107D1F43D
:149C9E00CC2021F481E090E07C0102C0EE24FF24EC82FE01FF
:149CB200EB54FD4F008011800A821B828EE39DE088839983C4
:149CC60025EB3CE001E41BE0E6D1D6C18AE090E0888399832F
:149CDA002AE430E28A010E9435E400300107D1F48AE390E234
:149CEE008C839D83CC2021F481E090E07C0102C0EE24FF24ED
:149D0200EA82FE01EB54FD4F008011800882198220EA35E4FE
:149D16000EE310E260D2B0C180E18093302F22E7CA01019675
:149D2A00AC018C010E945B3678010030010709F06FC028E3D4
:149D3E0030E28A010E94D6E2FE01E256FD4F0083118388E018
:149D520090E088839983FE01E256FD4F208131818E010056AB
:149D66001D4F0E9478E424E330E2002711270E94D6E2FE01AE
:149D7A00E256FD4F0083118383E090E088839983FE01E25609
:149D8E00FD4F208131818E0108551D4F0E9478E49E012855B0
:149DA2003D4F8E0100561D4F0E94E0370F3FEFEF1E07C9F409
:149DB600CC2019F441E050E002C0442755274C83FE01EB5499
:149DCA00FD4F008011800A821B8284E59DE08883998323ECE3
:149DDE003CE00AE51BE05BD12BC0CC2019F441E050E002C048
:149DF200442755274C83FE01EB54FD4F008011800A821B82E3
:149E060086EC9DE0888399832FEF3CE007EB1BE042D112C026
:149E1A00FE01EB54FD4F00801180088219829701CC2021F4DB
:149E2E0081E090E06C0102C0CC24DD240C2D8ED2222420929E
:149E4200302F1CC184E090E0888399832EE230E285010E948B
:149E560035E40030010709F0F1C022242A82CE010696888395
:149E6A00998329E832E0FE01EB54FD4F008111810E94F495DD
:149E7E00B8010030010709F4D3C0CE010696FB013197E80F29
:149E9200F91F20803324C1018D30E0E09E0729F08A30E0E036
:149EA6009E0709F0C1C0CE010696FB013297E80FF91F2080AA
:149EBA003324C1018D30E0E09E0729F08A30E0E09E0709F028
:149ECE00AFC081E08A83CE0106968883998329E832E0FE01EF
:149EE200EB54FD4F008111810E94C295B801CE010696FB01B5
:149EF600E80FF91F222420828FE090E0888399832EE130E23A
:149F0A008E010A5F1F4F0E9435E40030010769F4CE018057E7
:149F1E009D4F888399832BE030E28E010A5F1F4F0E946AE6A7
:149F32001AC08FE090E0888399832BEF3FE18E010A5F1F4F9B
:149F46000E9435E40030010761F4CE0180579D4F8883998306
:149F5A0028EE3FE18E010A5F1F4F0E946AE66230E0E07E078E
:149F6E0009F05BC0AA2009F458C0FE01E057FD4F2080318019
:149F8200222019F4332009F44EC088E892E08215930598F481
:149F960081E08C83FE01EB54FD4F008011800A821B828FE60E
:149FAA009DE08883998321ED3CE003E71BE071D061C0222448
:149FBE002A82CE01069688839983FE01E057FD4F208131817C
:149FD200FE01EB54FD4F008111810E949095B801FE01E05728
:149FE600FD4F208031800215130509F045C0CE010696FB0136
:149FFA00E80FF91F22242082CE010696FB013196E80FF91F1F
:14A00E00222420829E012A5F3F4FFE01EB54FD4F0081118103
:14A022000E94615B2BC0AA24A39405C06A38E2E07E0721F518
:14A03600AA246030670709F010CF1EC0CE0106968883998302
:14A04A009B01FE01EB54FD4F008111810E94DD9481E08C8346
:14A05E00FE01EB54FD4F008011800A821B8283EA9DE0888335
:14A0720099832BEE3CE008E91BE00FD0EF96EF96EF96EF96AA
:14A08600EF96EF96EF96EF96EF96EF96E5960E9411E02296E2
:14A09A0008950E94FCDFB90158012E974E895F89088C00204D
:14A0AE0009F45DC085010E94F97EA882B98298018A010E94BA
:14A0C2000E978AED9BE08883998321E230E08A010E940E97E7
:14A0D6008CE09CE0888399832FE030E08A010E940E978BE10A
:14A0EA009CE0888399832CE030E08A010E940E978BEF9BE0DC
:14A0FE008883998321E130E08A010E940E978B010E94F97E9E
:14A1120018010C891D892F923F920E94F97E9F918F918C5B03
:14A126009F4F5C01A00EB11EA882B98224EE3FE18E010E5FCA
:14A13A001F4F0E942BE38E010E5F1F4F0E9426E5CE01029675
:14A14E008883998398018A010E949A9689E59CE088839983CF
:14A1620025E030E08A010E940E978EE59CE08883998328E1E3
:14A1760030E08A010E940E978B010E94F97E688379839801CE
:14A18A008A010E940E9786E79CE0888399832CE130E08A0137
:14A19E000E940E970C891D890E94F97E18010C881D88088236
:14A1B200198291018A010E940E9782E99CE08883998323E188
:14A1C60030E08A010E940E978A010E94AF972E960E940BE0DF
:14A1DA0008950E9400E0B90158012E974E895F89088C002007
:14A1EE0009F480C084E19BE08883998322E130E08A010E94D9
:14A202000E978AED9BE08883998321E230E08A010E940E97A5
:14A216008CE09CE0888399832FE030E08A010E940E9783E0D1
:14A22A0090E08883998320EE3FE10A8D1B8D0E9435E4003031
:14A23E00010751F48BE19CE0888399832CE030E08A010E9467
:14A252000E9716C083E090E0888399832AE330E20A8D1B8D25
:14A266000E9435E40030010749F487E29CE0888399832DE09B
:14A27A0030E08A010E940E978BEF9BE08883998321E130E0C0
:14A28E008A010E940E9785010E9426E518018B012F923F9280
:14A2A2000E9426E59F918F918C5B9F4F6C01C00ED11EC88262
:14A2B600D98224EE3FE18E010E5F1F4F0E942BE38E010E5FF1
:14A2CA001F4F0E9426E5CE0102968883998398018A010E9411
:14A2DE009A9689E59CE08883998325E030E08A010E940E9744
:14A2F2008EE59CE08883998328E130E08A010E940E978501D1
:14A306000E9426E5A882B98298018A010E949A9686E79CE052
:14A31A00888399832CE130E08A010E940E978B010E9426E5E0
:14A32E006883798398018A010E949A9682E99CE08883998330
:14A3420023E130E08A010E940E978A010E94AF972E960E9448
:14A356000EE008950E94FCDFA901A02E2E976C897D89AA20E9
:14A36A0009F4DDC0AA2412C0CA010896EA2DFF27E80FF91FF0
:14A37E00008111270E94717ECE010296EA2DFF27E80FF91FCE
:14A392000083A3948A2D833058F384E19BE08883998322E13E
:14A3A60030E08B010E940E978AED9BE08883998321E230E094
:14A3BA008B010E940E978CE09CE0888399832FE030E08B0102
:14A3CE000E940E9783E090E08883998320EE3FE18E010E5F10
:14A3E2001F4F0E9435E40030010751F48BE19CE088839983B2
:14A3F6002CE030E08B010E940E9769C083E090E08883998341
:14A40A002AE330E28E010E5F1F4F0E9435E40030010751F47D
:14A41E0087E29CE0888399832DE030E08B010E940E9751C01D
:14A4320083E090E0888399832CED3FE18E010E5F1F4F0E94D7
:14A4460035E40030010751F481E49CE0888399832CE030E048
:14A45A008B010E940E9739C083E090E08883998328ED3FE1F3
:14A46E008E010E5F1F4F0E9435E40030010751F484E39CE055
:14A48200888399832DE030E08B010E940E9721C083E090E0FB
:14A496008883998324ED3FE18E010E5F1F4F0E9435E4003005
:14A4AA00010751F48DE49CE0888399832CE030E08B010E94F3
:14A4BE000E9709C08DE49CE0888399832CE030E08B010E94BE
:14A4D2000E978BEF9BE08883998321E130E08B010E940E97D0
:14A4E600CE01029688839983FA0100891189228933890E94AD
:14A4FA00923D8E010E5F1F4F0E9426E5CE01029688839983DA
:14A50E0098018B010E949A9689E59CE08883998325E030E01C
:14A522008B010E940E978FE599E3FB01E081FF27EE0FFF1FC4
:14A53600EE0FFF1FEE0FFF1FE80FF91FDB0111962D903C90C0
:14A54A002082318281E699E3FB01E081FF27EE0FFF1FEE0F2A
:14A55E00FF1FEE0FFF1FE80FF91FDB0113962D903C902082F1
:14A5720031828DE599E3FB01E081FF27EE0FFF1FEE0FFF1F7B
:14A58600EE0FFF1FE80FF91FDB0115962D903C902082318232
:14A59A0083E699E3FB01E081FF27EE0FFF1FEE0FFF1FEE0F12
:14A5AE00FF1FE80FF91F408351832E960E940BE008950E9445
:14A5C200E1DFA8012297FA01008111270E94717EFA010083A0
:14A5D600CA010196FC01008111278F939F930E94717EFF91E4
:14A5EA00EF910083CA010296FC01008111278F939F930E944B
:14A5FE00717EFF91EF91008383E090E08883998320EE3FE19F
:14A612008A010E9435E40030010719F40BE11CE03EC083E060
:14A6260090E0888399832AE330E28A010E9435E400300107EC
:14A63A0019F407E21CE02FC083E090E0888399832CED3FE1F8
:14A64E008A010E9435E40030010719F401E41CE020C083E049
:14A6620090E08883998328ED3FE18A010E9435E4003001079A
:14A6760019F404E31CE011C083E090E08883998324ED3FE1E4
:14A68A008A010E9435E40030010719F40DE41CE002C007E299
:14A69E001CE022960E94E4DF08950E94F8DFA8012597662787
:14A6B20019F461E070E002C0662777276C834A835B8384E506
:14A6C6009DE0888399832FEF3CE007EB1BE0E3DC25960E9499
:14A6DA0008E008950E94FCDFA90158012397B5016E5D7F4F5E
:14A6EE00FB0180819181892F992790708830E0E09E0709F5B6
:14A702001B016E5F7F4F44245524F101408251822224332487
:14A71600FB01208231829A0185010E5D1F4F0E94A555FB014C
:14A72A000083118381E08A830B841C840882198229853A85D5
:14A73E008A010E94A65323960E940BE008950E94FCDFB901C7
:14A75200A80124978DE799E35C014C5E5F4F80E095E4F5011B
:14A7660086879787408B518B2090952030909620C1010196D9
:14A77A009093962080939520228A338A22243324248A358AB7
:14A78E008C8599279064868B978B2224208E318E20900A3022
:14A7A20030900B30228E338E20900C3030900D30248E358ED9
:14A7B600668F778F0A841B8400A211A224E130E00BE819E30E
:14A7CA00BFD110939639009395390A841B840A821B826883D7
:14A7DE00798320E038E08A010E948C3224960E940BE0089584
:14A7F2000E9404E0B80128978DE799E35C0140918B39509192
:14A806008C39452F55274F705070440F551FFC01E05BFF4FBD
:14A81A00E080F180CC2422C02090733F3090743F222011F46B
:14A82E00332039F0C10101979093743F8093733F12C022248D
:14A84200332430926C3F20926B3F30926E3F20926D3F309253
:14A85600703F20926F3F3092723F2092713FC3948C2D823048
:14A86A00D8F29A01220F331F0BE819E369D10030010709F098
:14A87E0038C120900A3030900B30F501468C578C4214530490
:14A8920049F420900C3030900D3040A051A04214530489F095
:14A8A600F501868D978DEA938F3FEFEF9E07E99109F01BC154
:14A8BA0080A191A18F3FEFEF9E0709F014C1F501608971893F
:14A8CE00848995899F738030890709F4ADC02288338840905A
:14A8E2006B3F50906C3F2414350431F0222009F0A1C03320AC
:14A8F60009F09EC0F5012288338830926C3F20926B3F228C25
:14A90A00338C30926E3F20926D3F248C358C3092703F209219
:14A91E006F3F8689978990709093723F8093713F8AE090E0D7
:14A932009093743F8093733F1B0136942794241A350AC70190
:14A94600820D931D8033E2E09E0718F5CC24DD2418C0FA01D3
:14A95A003796EC0DFD1DEE0FFF1FEA0DFB1D20803180F70196
:14A96E00EC0DFD1DEE0FFF1F85E79FE3E80FF91F2082318255
:14A98200C60101966C011B0136942794241A350AC214D3042B
:14A9960000F3F5012488358835FC45C020908D3930908E3928
:14A9AA00648975897F71660F771F660F771F660F771F620D2E
:14A9BE00731D22243324248A358ACC24DD2416C0FA0137965C
:14A9D200EC0DFD1DEE0FFF1FEA0DFB1D85E79FE3D601AA0FB6
:14A9E600BB1FA80FB91F2D903C9020823182C60101966C014B
:14A9FA001B0136942794C214D30420F32224332430926C3FDE
:14AA0E0020926B3F30926E3F20926D3F3092703F20926F3F3A
:14AA22003092723F2092713F05C022243324F501268A378A82
:14AA3600F501868997899070EA938130E0E09E07E99199F44D
:14AA4A00248C358C2A823B82228C338C288239821A01220C03
:14AA5E00331C9B01221933090DE719E30E946F5369C0F5010F
:14AA7200868997899070EA938630E0E09E07E99179F4248C72
:14AA8600358C28823982228D338D1A01220C331C8B010219E8
:14AA9A0013090E94008050C0F501868997899070EA93813106
:14AAAE00E0E09E07E99109F045C020A031A02E823F82268C03
:14AAC200378C2C823D82248C358C2A823B82228C338C28825F
:14AAD60039821A01220C331C9B01221933098A01095F1F4FA5
:14AAEA000E94DC7329C020909420222029F1F5018689978999
:14AAFE009070EA938131E0E09E07E991D9F420A031A02E8228
:14AB12003F82268C378C2C823D82248C358C2A823B82228C04
:14AB2600338C288239821A01220C331C9B01221933098A01C1
:14AB3A00095F1F4F0E94DC7328960E9411E008950E94FCDFD5
:14AB4E00249740E050E060E070E0FE014083518362837383E7
:14AB6200AA24BB2418C018010E5F1F4FF101208031804424BB
:14AB76005524FE016080718082809380620C731C841C951C1F
:14AB8A006082718282829382C50101965C0119013694279470
:14AB9E00A214B30410F320FF14C0F8018081918180701C0127
:14ABB20044245524FE016080718082809380620C731C841C2C
:14ABC600951C60827182828293824FEF5FEF60E070E0FE01C1
:14ABDA002080318042805380242C352C442455242422352252
:14ABEE00462257224FEF5FEF60E070E0608071808280938070
:14AC02006422752286229722620C731C841C951C608271829D
:14AC16008282938240E050E06FEF7FEF20803180428053800F
:14AC2A00242235224622572240E050E060E070E02416350643
:14AC3E004606570681F041E050E060E070E0208031804280F4
:14AC52005380240E351E461E571E20823182428253824FEF91
:14AC66005FEF60E070E0FE012080318042805380242235227A
:14AC7A00462257222094309440945094810124960E940BE0EC
:14AC8E0008952C9744275527662781E08093D9432224209256
:14ACA200D8432092D74320926D0087E787BB88B38D6088BB7D
:14ACB60086EA82B983B1806A83B98FE681BB8FEF82BB80E5B4
:14ACCA008DB985B7806C85BF81E487BF80E189BF8FEF88BFAB
:14ACDE0083E08ABF23E934EA0AEC11E80E9455E8019904C060
:14ACF20081E08093A84603C022242092A846029909C100E0FE
:14AD060014E00E94F231580128E531E20E9485E300300107C5
:14AD1A0089F0950107EE16E40E947CEA27EE36E400E113E01C
:14AD2E000E94D33128E531E207EE16E40E947CEA00EC12E076
:14AD42000E94F231580128E531E20E9485E30030010789F004
:14AD560095010BEF16E40E947CEA2BEF36E400EC12E00E94A3
:14AD6A00D33128E531E20BEF16E40E947CEA00E012E00E9441
:14AD7E00B93110930B3000930A3002E012E00E94B931109329
:14AD92000D3000930C3080910A3090910B30883AE0EC9E07C7
:14ADA60041F480910C3090910D308E3FE0E09E07E1F088EA44
:14ADBA0090EC90930B3080930A308EEF90E090930D308093FE
:14ADCE000C3020910A3030910B3000E012E00E949331209165
:14ADE2000C3030910D3002E012E00E94933104E012E00E9471
:14ADF600B93110930F3000930E3006E012E00E94B9311093A5
:14AE0A0011300093103020900E3030900F30222051F4332059
:14AE1E0041F42090103030901130222011F43320D1F0222459
:14AE3200332430920F3020920E30309211302092103020911E
:14AE46000E3030910F3004E012E00E949331209110303091CC
:14AE5A00113006E012E00E94933108E012E00E94B93110935C
:14AE6E001730009316300AE012E00E94B931109319300093C9
:14AE820018302090163030901730222051F4332041F42090B8
:14AE9600183030901930222011F43320D1F02224332430929D
:14AEAA00173020921630309219302092183020911630309198
:14AEBE00173008E012E00E94933120911830309119300AE00C
:14AED20012E00E94933123E300E214E00E948231222701E2B7
:14AEE60014E00E94823123E002E214E00E948231222703E2B1
:14AEFA0014E00E94823103E30E94E0712224288223E0002708
:14AF0E000E94FE710E94C673069906C081E080937E278093B2
:14AF22006D730BC0222420927E27059903C020926D7303C01D
:14AF360081E080936D7322242092F04381E08093E74304994D
:14AF4A0003C08093F14303C022242092F1430E94A624222448
:14AF5E002092302F2092312FC59AC49A0E9491350E940D9850
:14AF720087E083BF85E085BD78940E94077A0130A9F480E11D
:14AF86008093302F22242092312F0E94D53A03990BC00E9433
:14AF9A00FD790E94A99F002301F022242092302F2092312FC6
:14AFAE008AEF8093E84380E18093302F8093312F2090E843B7
:14AFC200222021F081E090E06C0102C0CC24DD2486B3807806
:14AFD600803821F481E090E05C0102C0AA24BB2416012A209C
:14AFEA003B20222039F7332029F722242092302F2092312FAA
:14AFFE00B7990BC02090F143222019F00E94CA2902C00E94FC
:14B0120063350E940F4C2090D743222041F020916C25009185
:14B02600D9430E9419D10093D843019904C081E08093A84600
:14B03A0003C022242092A846069906C081E080937E278093C8
:14B04E006D730BC0222420927E27059903C020926D7303C0F0
:14B0620081E080936D732090EB433090D543321409F416C1B6
:14B0760000E80E944F5B0093EB4302E80E944F5B0093EA43DB
:14B08A0004E80E944F5B0093E9430CE80E944F5B0093EC43B9
:14B09E0008E80E944F5B0093ED4306E80E944F5B0093EF43A0
:14B0B2000AE80E944F5B0093EE432090EB432092D543209030
:14B0C600D743222009F451C0E090D843C090E94388ED93E419
:14B0DA008883998320916C250091D9430E94F1CFC02E20904C
:14B0EE00D843E21429F0222D07E314E00E9482312090E943C6
:14B10200C214A9F1C092E9432090EB43332428823982209100
:14B11600EA4333270C2D11270E94DA5A2090D843222091F0C9
:14B12A008091D943813029F40CE311E20E94CFE51AC08091F3
:14B13E00D9438230B1F400E211E20E94CFE511C08091D94361
:14B15200813029F403E011E20E94CFE508C08091D943823048
:14B1660021F406EE10E20E94CFE5222430909A20231420F479
:14B17A00832D815080939A2020909A202220D9F52090EB431B
:14B18E00222021F020905F25222099F12090E943222021F427
:14B1A2002090EA43222031F020905F252220E9F04423D9F4D6
:14B1B60022E70AED13E40E945B3610937330009372300030B0
:14B1CA00010779F00E943F3A21E00AED13E40E94477C602F02
:14B1DE00063920F00C3B11F00E942B3241E00091EB430E9445
:14B1F2005EC3602F86E9081710F00E942B322090A84622202C
:14B2060029F42090A946222009F448C080916D73813031F569
:14B21A002090EB4333242A863B862090EA43332428863986D9
:14B22E002090E94333242E823F822090EE4333242C823D82C3
:14B242002090EC4333242A823B822090EF43332428823982BB
:14B256002091ED43332700EC10E20E94CFE51EC02091ED43B6
:14B26A0009E10E9442232091EF430AE10E9442232091EC432A
:14B27E000BE10E9442232091E9430CE10E9442232091EA431A
:14B292000DE10E9442232091EB430EE10E9442230E94534C9D
:14B2A6000E94193E80919820813009F05AC0A0906D73BB241F
:14B2BA0081E080936D7322242092982022E707EB10E20E94ED
:14B2CE005B36109373300093723000300107D1F000919B201B
:14B2E20010919C200E94A4230A3A31F40091723010917330B2
:14B2F6000E94DA2300917230109173300E943F3A07EB10E22F
:14B30A000E94173BA0926D7322E70AEA10E20E945B36109364
:14B31E0073300093723000300107F9F00E943F3A0DE910E21F
:14B332000E94173B2DE930E20AED13E40E9465392AED33E48F
:14B346000AEA10E20E94653921E00AED13E40E94477C602FEA
:14B35A00063920F00C3B11F00E942B3241E080916D73813086
:14B36E0091F420909920222039F020907E27222019F40E942C
:14B382009C7618C00E94C2140023A1F00E94331511C0209036
:14B396006D73222069F420908528222049F0209099202220A1
:14B3AA0019F00E949C7602C00E94D9220E94077A013009F026
:14B3BE0038CEE090302F80E18093302FC090312F222420922B
:14B3D200312F0E94D53AE092302FC092312F27CE2C9608957F
:14B3E6000E9484DF0E94F8DFB79904C00E94092E0E940B8FAC
:14B3FA002090E843222029F08091E84381508093E84320900E
:14B40E008581222029F08091858181508093858100E80E943E
:14B422004F5B0093EB432090D64320942092D6433090312F43
:14B4360032204091302F4325407366B36F7C262E242A28BADD
:14B44A00222422BE0E9408E00E949BDF18950E9484DF0E94CE
:14B45E00E1DFB7991FC0409124F1509125F14430E0E05E0775
:14B4720019F480E884BD14C050FD0FC0409102F4509103F481
:14B48600409102F1509103F1509303F1409302F180E884BDD3
:14B49A0003C00E94F633E1CF0E94E4DF0E949BDF18950E9490
:14B4AE00E1DF4091D84320916C250091D9430E9419D10093D0
:14B4C200D843202E401729F0222D07E314E00E9482310E9479
:14B4D600E4DF08950E9400E0422FC02E5FD08D9A8C9894987B
:14B4EA004E7FAA240CC0042F1A2D0E9401EB602F617011F07E
:14B4FE00959A01C0959854D0A39487E08A1588F74C2DAA24F6
:14B512000CC0042F1A2D0E9401EB602F617011F0959A01C000
:14B52600959842D0A39487E08A1588F70E940EE008950E9447
:14B53A0000E0602F442730D08D9A8C9894986160AA240EC04F
:14B54E00062F1A2D0E9401EB802F8170C82E882311F0959A6E
:14B5620001C0959823D0A39487E08A1578F78D988C989498D3
:14B57600AA240DC060B3862F82958F708170682F082F1A2D42
:14B58A000E94FBEA402B0ED0A39487E08A1580F7042F0E9454
:14B59E000EE008951A98959A949896981A9A0895969A969824
:14B5B20008950E94FCDFA22E402F1AE0042F0E949E7E602FB2
:14B5C6001AE0042F0E949C7E402F862F8F708295482B4F7319
:14B5DA0024E8042F7DDF1AE00A2D0E949E7E602F1AE00A2D13
:14B5EE000E949C7E402F862F8F708295482B22E8042F6CDF58
:14B602001AE00E810E949E7E602F1AE00E810E949C7E402FAA
:14B61600862F8F708295482B20E8042F5BDF0E940BE0089543
:14B62A000E9400E0A22EC02E1AE008850E949E7E602F1AE0FE
:14B63E0008850E949C7E402F862F8F708295482B2CE8042FBB
:14B6520043DF1AE00C2D0E949E7E602F1AE00C2D0E949C7E53
:14B66600402F862F8F708295482B28E8042F32DF1AE00A2D9E
:14B67A000E949E7E602F1AE00A2D0E949C7E402F862F8F705F
:14B68E008295482B26E8042F21DF0E940EE008950E94F8DF37
:14B6A200402F042F48DF402F642F607F62956F708AE0869F85
:14B6B6004F70400D042F0E9408E008950E94F8DFB901A8013E
:14B6CA0026972224209298450EC086EF93E4E0919845FF27AC
:14B6DE00E80FF91F22242082809198458F5F80939845809184
:14B6F20098458F3F70F322242092984517C08FE795E4E0912A
:14B706009845FF27E80FF91F222420828BE695E4E0919845FD
:14B71A00FF27E80FF91F22242082809198458F5F8093984532
:14B72E0080919845843128F322242092984520926B45209260
:14B742007F4520929F4520929E45222433243092F5432092BB
:14B75600F44370936A4560936945709368456093674569C0DD
:14B76A00E0916745F09168458081853279F5CF0101969093D0
:14B77E0068458093674582E090E08883998320916745309134
:14B7920068450BE615E40E9485EA81E090E08883998321EEF4
:14B7A60034E20DE615E40E9485EA0BE615E40E94AB4BE09189
:14B7BA006945F0916A450083809167459091684502969093D4
:14B7CE006845809367452AC0E0916745F091684580818B3208
:14B7E20081F480E2E0916945F0916A4580838091674590914C
:14B7F60068450196909368458093674513C0E0916745F091FB
:14B80A0068452080E0916945F0916A4520828091674590910E
:14B81E006845019690936845809367458091694590916A45B4
:14B83200019690936A4580936945E0916745F09168452080ED
:14B84600222041F0CF01861B970B8A38E2E09E0708F488CFEC
:14B85A002224E0916945F0916A4520822FED34E28B010E9443
:14B86E00D6E21093F3430093F2435CC42DED34E200271127BE
:14B882000E94D6E21093FB440093FA4428ED34E20091F243B4
:14B896001091F3430E9485E30030010729F46091FA44709138
:14B8AA00FB4438C42FEC34E20091F2431091F3430E9485E377
:14B8BE000030010729F46091FA447091FB4428C42BEC34E299
:14B8D2000091F2431091F3430E9485E30030010749F4209096
:14B8E600FA443090FB44309253452092524514C425EC34E26F
:14B8FA000091F2431091F3430E9485E30030010749F420906E
:14B90E00FA443090FB44309255452092544500C421EC34E25A
:14B922000091F2431091F3430E9485E30030010749F4209045
:14B93600FA443090FB443092574520925645ECC32CEB34E239
:14B94A000091F2431091F3430E9485E30030010749F420901D
:14B95E00FA443090FB443092594520925845D8C326EB34E227
:14B972000091F2431091F3430E9485E30030010749F42090F5
:14B98600FA443090FB4430925B4520925A45C4C32EEA34E208
:14B99A000091F2431091F3430E9485E30030010749F42090CD
:14B9AE00FA443090FB4430925D4520925C45B0C326EA34E2F8
:14B9C2000091F2431091F3430E9485E30030010749F42090A5
:14B9D600FA443090FB4430925F4520925E459CC320E934E2E7
:14B9EA000091F2431091F3430E9485E30030010721F481E0F4
:14B9FE0080939F458DC325E834E20091F2431091F3430E948C
:14BA120085E30030010721F481E080939E457EC32AE734E2AC
:14BA26000091F2431091F3430E9485E30030010749F4209040
:14BA3A00FA443090FB4430920B4520920A456AC32FE634E250
:14BA4E000091F2431091F3430E9485E30030010749F4209018
:14BA6200FA443090FB4430920D4520920C4556C324E634E243
:14BA76000091F2431091F3430E9485E30030010749F42090F0
:14BA8A00FA443090FB4430920F4520920E4542C329E534E227
:14BA9E000091F2431091F3430E9485E30030010749F42090C8
:14BAB200FA443090FB4430921145209210452EC329E434E210
:14BAC6000091F2431091F3430E9485E30030010749F42090A0
:14BADA00FA443090FB4430921345209212451AC329E334E2F9
:14BAEE000091F2431091F3430E9485E30030010749F4209078
:14BB0200FA443090FB44309215452092144506C329E234E2E1
:14BB16000091F2431091F3430E9485E30030010749F420904F
:14BB2A00FA443090FB443092174520921645F2C229E134E2CB
:14BB3E000091F2431091F3430E9485E30030010749F4209027
:14BB5200FA443090FB443092194520921845DEC22DE034E2B0
:14BB66000091F2431091F3430E9485E30030010749F42090FF
:14BB7A00FA443090FB4430921B4520921A45CAC221E034E2A4
:14BB8E000091F2431091F3430E9485E30030010749F42090D7
:14BBA200FA443090FB4430921D4520921C45B6C225EF33E27A
:14BBB6000091F2431091F3430E9485E30030010749F42090AF
:14BBCA00FA443090FB4430921F4520921E45A2C229EE33E25F
:14BBDE000091F2431091F3430E9485E30030010749F4209087
:14BBF200FA443090FB4430922145209220458EC226ED33E24B
:14BC06000091F2431091F3430E9485E30030010749F420905E
:14BC1A00FA443090FB4430922345209222457AC22CEC33E22D
:14BC2E000091F2431091F3430E9485E30030010749F4209036
:14BC4200FA443090FB44309225452092244566C22BEB33E217
:14BC56000091F2431091F3430E9485E30030010749F420900E
:14BC6A00FA443090FB44309227452092264552C22AEA33E201
:14BC7E000091F2431091F3430E9485E30030010749F42090E6
:14BC9200FA443090FB4430922945209228453EC229E933E2EB
:14BCA6000091F2431091F3430E9485E30030010749F42090BE
:14BCBA00FA443090FB4430922B4520922A452AC228E833E2D5
:14BCCE000091F2431091F3430E9485E30030010749F4209096
:14BCE200FA443090FB4430922D4520922C4516C22CE733E2BA
:14BCF6000091F2431091F3430E9485E30030010749F420906E
:14BD0A00FA443090FB4430922F4520922E4502C22BE633E2A3
:14BD1E000091F2431091F3430E9485E30030010721F481E0BC
:14BD320080936645F3C122E633E20091F2431091F3430E942F
:14BD460085E30030010749F42090FA443090FB4430923145E7
:14BD5A0020923045DFC129E533E20091F2431091F3430E94AC
:14BD6E0085E30030010749F42090FA443090FB4430923345BD
:14BD820020923245CBC12BE433E20091F2431091F3430E9495
:14BD960085E30030010749F42090FA443090FB443092414587
:14BDAA0020924045B7C12DE333E20091F2431091F3430E9472
:14BDBE0085E30030010749F42090FA443090FB44309243455D
:14BDD20020924245A3C120E333E20091F2431091F3430E9469
:14BDE60085E30030010749F42090FA443090FB443092354543
:14BDFA00209234458FC124E233E20091F2431091F3430E9460
:14BE0E0085E30030010749F42090FA443090FB443092374518
:14BE2200209236457BC12AE133E20091F2431091F3430E9444
:14BE360085E30030010749F42090FA443090FB4430923945EE
:14BE4A002092384567C121E133E20091F2431091F3430E9437
:14BE5E0085E30030010749F42090FA443090FB4430923B45C4
:14BE720020923A4553C128E033E20091F2431091F3430E941B
:14BE860085E30030010749F42090FA443090FB4430923D459A
:14BE9A0020923C453FC12CEF32E20091F2431091F3430E94F3
:14BEAE0085E30030010749F42090FA443090FB44309245456A
:14BEC200209244452BC120EF32E20091F2431091F3430E94E3
:14BED60085E30030010749F42090FA443090FB443092474540
:14BEEA002092464517C12BEE32E20091F2431091F3430E94C3
:14BEFE0085E30030010749F42090FA443090FB443092FD4463
:14BF12002092FC4403C123EE32E20091F2431091F3430E9401
:14BF260085E30030010749F42090FA443090FB443092FF4438
:14BF3A002092FE44EFC02BED32E20091F2431091F3430E94E5
:14BF4E0085E30030010749F42090FA443090FB44309201450D
:14BF620020920045DBC024ED32E20091F2431091F3430E94D5
:14BF760085E30030010749F42090FA443090FB4430920545E1
:14BF8A0020920445C7C025EC32E20091F2431091F3430E94BD
:14BF9E0085E30030010749F42090FA443090FB443092F543CB
:14BFB2002092F443B3C02AEB32E20091F2431091F3430E94B7
:14BFC60085E30030010749F42090FA443090FB44309249454D
:14BFDA00209248459FC020EB32E20091F2431091F3430E9457
:14BFEE0085E30030010749F42090FA443090FB443092094565
:14C00200209208458BC02BEA32E20091F2431091F3430E9478
:14C0160085E30030010749F42090FA443090FB4430924B45FA
:14C02A0020924A4577C022EA32E20091F2431091F3430E942B
:14C03E0085E30030010749F42090FA443090FB4430924D45D0
:14C0520020924C4563C029E932E20091F2431091F3430E940F
:14C0660085E30030010749F42090FA443090FB4430924F45A6
:14C07A0020924E454FC022E932E20091F2431091F3430E9400
:14C08E0085E30030010749F42090FA443090FB44309251457C
:14C0A200209250453BC029E832E20091F2431091F3430E94E4
:14C0B60085E30030010749F42090FA443090FB443092614544
:14C0CA002092604527C020E832E20091F2431091F3430E94C9
:14C0DE0085E30030010749F42090FA443090FB44309263451A
:14C0F2002092624513C02AE732E20091F2431091F3430E94AA
:14C1060085E30030010741F42090FA443090FB4430926545F7
:14C11A00209264452FED34E2002711270E94D6E21093F343F2
